:020000040800F2
:1000000000070020F1010008152D0008CD2C000884
:10001000F52C0008CD2C0008ED2C0008F301000899
:10002000F3010008F3010008F3010008093D00088E
:10003000F3010008F3010008F3010008F3010008D0
:10004000F3010008F3010008F3010008F3010008C0
:10005000F3010008F3010008A1620008C96200086A
:10006000F16200081963000841630008F301000809
:10007000F3010008F3010008F3010008F301000890
:10008000F3010008F3010008F30100085D2C0008EB
:100090006D2C0008812C0008F3010008696300083A
:1000A000F3010008F3010008F3010008F301000860
:1000B0003D640008F3010008F3010008F3010008A3
:1000C000F3010008F3010008F3010008F301000840
:1000D000F3010008F3010008F3010008F301000830
:1000E000CD630008F3010008F3010008F3010008E4
:1000F000F3010008F3010008F3010008F301000810
:10010000F3010008F3010008F3010008F3010008FF
:10011000F3010008F3010008F3010008F3010008EF
:10012000F3010008F3010008F3010008F3010008DF
:10013000F3010008F3010008F3010008952C000802
:10014000A52C0008B92C0008F301000895580008F8
:10015000F3010008F3010008F3010008F3010008AF
:10016000F3010008F3010008F3010008F30100089F
:10017000F3010008F3010008F3010008F30100088F
:10018000F3010008F3010008F3010008F30100087F
:10019000F3010008F3010008F3010008F30100086F
:1001A000F3010008F3010008F3010008F30100085F
:1001B000F3010008F3010008F3010008F30100084F
:1001C000F3010008F3010008F3010008F30100083F
:1001D000F3010008F3010008F3010008F30100082F
:1001E000C915000800000000000000000000000029
:1001F00002E000F000F8FEE772B6374880F30888A6
:10020000364880F3098836483649086040F20000D5
:10021000CCF200004EF63471CEF200010860BFF35C
:100220004F8FBFF36F8F40F20000C0F2F0004EF628
:100230008851CEF200010860BFF34F8FBFF36F8F7C
:100240004FF00000E1EE100A4EF63C71CEF20001D4
:100250000860062080F31488BFF36F8F04F0E2FF7C
:1002600005F0C6FE4FF055301F491B4A91423CBF76
:1002700041F8040BFAE71D49184A91423CBF41F886
:10028000040BFAE71A491B4A1B4B9A423EBF51F82E
:10029000040B42F8040BF8E700201849184A914271
:1002A0003CBF41F8040BFAE704F0C0FF05F0F4FE90
:1002B000144C154DAC4203DA54F8041B8847F9E797
:1002C00000F042F8114C124DAC4203DA54F8041B12
:1002D0008847F9E704F0A8BF0007002000230020AA
:1002E0000000000808ED00E00001002000070020E9
:1002F000186A000800230020B0230020B02300204B
:100300000C670020E0010008E4010008E401000897
:10031000E40100082DE9F04F2DED108AC1F80CD052
:10032000C3689D46BDEC108ABDE8F08F002383F3BF
:1003300011882846A047002004F078FAFEE704F070
:10034000F7F900DFFEE70000F8B501F0A7F904F0C7
:1003500003FF074604F052FF0546A8BB1F4B9F4210
:1003600032D001339F4232D01D4B27F0FF029A4218
:1003700030D1F8B200F034FF2E4642F2107400F093
:1003800035FF08B10024264601F034FD20B10320DA
:1003900000F07AF80024264635B1124B9F4203D074
:1003A00004F024FF00242646002004F0DFFE0EB1F6
:1003B00000F080F801F0CEFA00F084FF204600F053
:1003C000DFF800F077F8F9E72E460024D7E7044677
:1003D0000126D4E7064641F28834D0E7010007B091
:1003E000000008B0263A09B008B501F029F9A0F1DB
:1003F00020035842584108BD07B541F212030221BB
:1004000001A8ADF8043001F039F903B05DF804FB40
:1004100038B5302383F31188174803680BB104F013
:10042000D1FA164A144800234FF47A7104F0C0FA46
:10043000002383F31188124C236813B12368013B16
:100440002360636813B16368013B63600D4D2B78D3
:1004500033B963687BB9022001F0E6F932236360A7
:100460002B78032B07D163682BB9022001F0DCF94C
:100470004FF47A73636038BDB02300201104000884
:10048000D0240020C8230020084B187003280CD863
:10049000DFE800F008050208022001F0BBB90220E5
:1004A00001F0AEB9024B00225A607047C823002009
:1004B000D024002010B501F09DFC30B1294B03225F
:1004C0001A70294B00225A6010BD284B284A1C463E
:1004D00019680131F8D004339342F9D16268254B91
:1004E0009A42F1D9244B9B6803F1006303F58033F2
:1004F0009A42E9D204F04EFE04F060FE002001F0C2
:10050000E7F80220FFF7C0FF1C4B1A6C00221A64A8
:10051000196E1A66196E596C5A64596E5A665A6E7B
:100520005A6942F080025A615A6922F080025A6187
:100530005A691A6942F000521A611A6922F000528F
:100540001A611B6972B64FF0E0233021C3F8084DE1
:10055000D4E9003281F311889D4683F3088810475F
:10056000B2E700BFC8230020D0240020000001080B
:1005700020000108FFFF000800230020003802408F
:100580002DE9F04F93B0AC4B00902022FF210AA838
:100590009D6801F089F9A94A1378A3B9A8480121F7
:1005A00003601170302383F3118803680BB104F0EA
:1005B00009FAA44AA24800234FF47A7104F0F8F92A
:1005C000002383F31188009B13B19F4B009A1A609C
:1005D0009E4A009C1378032B1EBF002313709A4A77
:1005E0004FF0000A18BF5360D3465646D14601204B
:1005F00001F010F924B1944B1B68002B00F0158218
:10060000002001F01DF80390039B002B01DA00F09D
:10061000ABFE039B002BEDDB012001F0F1F8039B07
:10062000213B162BE3D801A252F823F089060008DB
:10063000B106000845070008EF050008EF050008AF
:10064000EF050008CF0700089F090008B908000857
:100650001B0900084309000869090008EF050008A4
:100660007B090008EF050008ED09000829070008CC
:10067000EF050008310A0008950600082907000860
:10068000EF0500081B0900080220FFF7ADFE002857
:1006900040F0F581009B0221BAF1000F08BF1C4613
:1006A00005A841F21233ADF8143000F0E7FF9EE7E1
:1006B0004FF47A7000F0C4FF071EEBDB0220FFF757
:1006C00093FE0028E6D0013F052F00F2DA81DFE833
:1006D00007F0030A0D10133605230593042105A81E
:1006E00000F0CCFF17E054480421F9E758480421F2
:1006F000F6E758480421F3E74FF01C08404600F0A5
:10070000E9FF08F104080590042105A800F0B6FFF0
:10071000B8F12C0FF2D1012000FA07F747EA0B0BD2
:100720005FFA8BFB4FF0000901F00AF926B10BF0DC
:100730000B030B2B08BF0024FFF75EFE57E746486C
:100740000421CDE7002EA5D00BF00B030B2BA1D17C
:100750000220FFF749FE074600289BD0012000F049
:10076000B7FF0220FFF790FE00261FFA86F84046EA
:1007700000F0BEFF044690B10021404600F0D0FFDB
:1007800001360028F1D1BA46044641F21213022183
:1007900005A8ADF814303E4600F070FF27E70120B1
:1007A000FFF772FE2546244B9B68AB4207D92846CB
:1007B00000F090FF013040F067810435F3E7234BF0
:1007C00000251D70204BBA465D603E46ACE7002E0A
:1007D0003FF460AF0BF00B030B2B7FF45BAF0220F9
:1007E000FFF752FE322000F02BFFB0F10008FFF6B9
:1007F00051AF18F003077FF44DAF0F4A926808EB32
:10080000050393423FF646AFB8F5807F3FF742AF0E
:10081000124B0193B84523DD4FF47A7000F010FFBE
:100820000390039A002AFFF635AF019B039A03F861
:10083000012B0137EDE700BF00230020CC2400206E
:10084000B023002011040008D0240020C823002079
:1008500004230020082300200C230020CC230020A8
:10086000C820FFF7C1FD074600283FF413AF1F2D36
:1008700011D8C5F1200242450AAB25F0030028BF7C
:10088000424683490192184400F0E8FF019A8048EB
:10089000FF2101F009F84FEAA8037D490193C8F34D
:1008A0008702284601F008F8064600283FF46DAF9D
:1008B000019B05EB830537E70220FFF795FD002834
:1008C0003FF4E8AE00F04CFF00283FF4E3AE002711
:1008D000B846704B9B68BB4218D91F2F11D80A9B92
:1008E00001330ED027F0030312AA134453F8203C1F
:1008F00005934046042205A901F034FA04378046E6
:10090000E7E7384600F0E6FE0590F2E7CDF8148000
:10091000042105A800F0B2FE06E70023642104A824
:10092000049300F0A1FE00287FF4B4AE0220FFF78C
:100930005BFD00283FF4AEAE049800F0F9FE059090
:10094000E6E70023642104A8049300F08DFE00284C
:100950007FF4A0AE0220FFF747FD00283FF49AAED7
:10096000049800F0F5FEEAE70220FFF73DFD0028BD
:100970003FF490AE00F004FFE1E70220FFF734FD02
:1009800000283FF487AE05A9142000F0FFFE0421E3
:100990000746049004A800F071FE3946B9E73220FA
:1009A00000F04EFE071EFFF675AEBB077FF472AE79
:1009B000384A926807EB090393423FF66BAE022078
:1009C000FFF712FD00283FF465AE27F003074F4400
:1009D000B9453FF4A9AE484600F07CFE04210590DD
:1009E00005A800F04BFE09F10409F1E74FF47A7015
:1009F000FFF7FAFC00283FF44DAE00F0B1FE0028EE
:100A000044D00A9B01330BD008220AA9002000F031
:100A100053FF00283AD02022FF210AA800F044FF0B
:100A2000FFF7EAFC1C4803F007FF13B0BDE8F08FA6
:100A3000002E3FF42FAE0BF00B030B2B7FF42AAEEE
:100A40000023642105A8059300F00EFE0746002848
:100A50007FF420AE0220FFF7C7FC804600283FF459
:100A600019AEFFF7C9FC41F2883003F0E5FE0598A6
:100A700000F098FF464600F063FF3C46B7E50646A7
:100A800052E64FF0000905E6BA467EE637467CE6B8
:100A9000CC23002000230020A0860100094A13680F
:100AA00049F2690099B21B0C00FB01331360064B3D
:100AB000186844F2506182B2000C01FB0200186019
:100AC00080B27047182300201423002010B50021A5
:100AD0001022044600F0E8FE034B03CB2060616067
:100AE0001868A06010BD00BF107AFF1F2DE9F0410B
:100AF000ADF54C7D0DF12C086AAC40F2751207463D
:100B00000D460CA80021C8F8001000F0CDFE4FF4EF
:100B1000C4720021204600F0C7FE02F003F9274B03
:100B20004FF47A72B0FBF2F0186093E807000223EA
:100B300084E807000DF5E5702382FFF7C7FF47F251
:100B400017031F49238407A805F088FD0F2384F8A5
:100B500032310DF2DB2207AB0DF1240C1E4603CE21
:100B6000664510605160334602F10802F6D13068E4
:100B70001060B188B379937191802046414601227B
:100B800000F012FF00230393AB7E029305F11903DB
:100B9000019380B20123CDE904800093E97E05A38F
:100BA000D3E90023384602F085FC0DF54C7DBDE805
:100BB000F08100BF9E6AC421818A46EED8240020BD
:100BC0006C6600082DE9F0412C4C237ADAB080469F
:100BD0000D465BBB27A9284600F0F6FF0746002814
:100BE00042D19DF89D60C82E3ED801464FF4A662C2
:100BF000204600F059FE4FF48073C4F8F8314FF4EA
:100C00000073C4F80C334FF44073C4F820343246F8
:100C10000DF19E0104F1090000F020FE26449DF82C
:100C20009C30777223720BB9EB7E237281220021F4
:100C300006AC27A800F038FE0122214627A800F0C4
:100C4000FFFF00230393AB7E029305F1190380B2EB
:100C500001932823CDE904400093E97E05A3D3E95D
:100C60000023404602F026FC5AB0BDE8F08100BFE8
:100C7000AFF3008026417272DF25D7B7D05600202F
:100C8000F0B5254E4FF48A7505FB0065F1B096F876
:100C9000D83085F8DC300024D822214685F8E84099
:100CA0003AA800F001FE06F1090000F0F5FDD5F8C4
:100CB000E4308DF8F000C2B206AF06F109010DF183
:100CC000F100CDE93A3400F0C9FD394601223AA8D5
:100CD00000F0E2FF80B2CDE9047008230127CDE9DE
:100CE000023706F1D803019330230093317A0B4881
:100CF00007A3D3E9002302F0DDFBA04206DD02F0EA
:100D000011F8C5F8E000384671B0F0BD2046FBE7A9
:100D100078F6339F93CACD8DD0560020F034002052
:100D20002DE9F04F274FDFF8A880274E87B03846CF
:100D300002F0ECFB034600283DD00024CDE903443B
:100D4000ADF81440027B8DF8142099684068029435
:100D500003AA03C21B681D4D43F000430293A14642
:100D6000A2462B68D3F810B001F0DEFF10EB0802AA
:100D700041F100032846CDF800A002A9D84704F2AB
:100D8000364440F66C030028C8BF49F0010905F558
:100D900086559C4205F11805E3D1B9F1000F05D045
:100DA000384602F0B7FB86F800A0C0E73378072B7F
:100DB00004D80133337007B0BDE8F08F014802F06A
:100DC000A9FBF8E7F0340020055C00202035002066
:100DD00040420F0070B50D4614461E4602F0C6FA9A
:100DE00050B9022E10D1012C0ED112A3D3E9002349
:100DF000C5E90023012007E0282C10D005D8012CDC
:100E000009D0052C0FD0002070BD302CFBD10BA3D6
:100E1000D3E90023ECE70BA3D3E90023E8E70BA316
:100E2000D3E90023E4E70BA3D3E90023E0E700BF05
:100E3000AFF30080401DA12026812A0B78F6339F56
:100E400093CACD8D9E6AC421818A46EE2641727274
:100E5000DF25D7B7F017304A39059E5638B5054615
:100E60000E4C0021013500F05BFCA4F82C55B4F8C1
:100E70002C0500F03DFC78B1B4F82C0500F048FCDE
:100E8000014648B9B4F82C0500F04AFCB4F82C35FA
:100E90000133A4F82C35EAE738BD00BFD056002056
:100EA000F8B50E4C0E4F0226A4F5805343F8487C4B
:100EB000237E3BB965692DB1284601F019F8284613
:100EC00005F00CFB204601F013F8A4F58654012E22
:100ED000A4F1180400D1F8BD0126E5E74056002032
:100EE000286700082DE9F04F8FB000AF05460C468B
:100EF00002F03CFA002849D1237E022B1BD1E38A61
:100F0000012B18D101F00EFF0646FFF7C7FD03467F
:100F10004FF4C870DFF8C482B3FBF0F206F5167622
:100F200002FB103316FA83F3C8F80030E37E33B9BE
:100F3000A34B00221A703C37BD46BDE8F08F07F185
:100F40002401204600F0FEFD0028F4D107F1140032
:100F5000FFF7BCFD97F8264007F11401224607F180
:100F6000270005F005FB0028E2D10F2C08D8944B90
:100F70001C70D8F80030A3F51673C8F80030DAE713
:100F800097F82410284602F0E9F9D4E7E38A282BE1
:100F90002BD010D8012B23D0052BCCD1BFF34F8FF2
:100FA0008849894BCA6802F4E0621343CB60BFF3FF
:100FB0004F8F00BFFDE7302BBDD1844EE17E327AEA
:100FC0009142B8D1607E3146002291F8DC508542D2
:100FD00000F0A5800132042A01F58A71F5D1AAE753
:100FE00021462846FFF782FDA5E721462846FFF760
:100FF000E9FDA0E7B2F8EC507B6005F103094FEA88
:1010000099094FEA8902D11DC908A8EBC1039D4681
:10101000EB460021584600F047FC04F1EE012A4659
:101020003144584600F01AFC7B6813B9012000F0E7
:101030004FFB96F8D20000F05BFB044630B93072EB
:1010400000F08EFB204600F043FBB1E0D6F8D42040
:101050003AB996F8D200B6F82C25824201D8FFF7AB
:10106000FDFED6F8D4202A44944208D296F8D20045
:10107000B6F82C250130824201D8FFF7EFFE7068E8
:101080005FFA89F2594600F017FC08B9C54679E0C5
:10109000726896F8D2002A447260D6F8D42005EB24
:1010A0000209C6F8D49000F023FB814509D396F8D5
:1010B000D220D6F8D4000132001B86F8D220C6F820
:1010C000D400FF2D0FD80024347200F049FB2046D5
:1010D00000F0FEFA00F08EFE3D4B188108B9FFF7D4
:1010E000E9F9C54627E7BB6896F8D9000AFB036211
:1010F000FB68D2F8E41082F8E83001F58061C2F8AC
:10110000E030C2F8E410FFF7BBFDFFF709FE96F8E8
:10111000D920013202F0030286F8D920B6E74FF455
:101120008A7A0AFB02F505F1EA013144204600F013
:10113000DFFDF86000287FF4FEAE3544012285F81B
:10114000E82001F0EFFDD5F8E020D6ED007ADFEDE4
:10115000216A801A192838BF192040F6B832904207
:1011600028BF1046B8EE677A07EE900AF8EEE77AE5
:1011700067EEA67ADFED186AE7EE267AFCEEE77AEC
:10118000C6ED007A96F8D930BB60BA6873680AFB7E
:1011900002F4321992F8E81059B1D2F8E4108B42F7
:1011A000E8463FF427AF002182F8E810C2F8E010CB
:1011B000C5467368064A9B0A01331381BBE600BF2C
:1011C000E934002000ED00E00400FA05D0560020CC
:1011D000D8240020CDCCCC3D6666663FEC340020A0
:1011E000014B1870704700BFE424002030B54FF069
:1011F00000542B4B22689A4285B007D004F008F8BF
:10120000044620BB0024204605B030BD254B627D3E
:1012100025481A70237D03724FF48073C0F8F831AB
:101220004FF40073C0F80C3300254FF44073C0F83E
:1012300020341E49C0F8E450C922093000F00EFBEA
:101240002046E022294600F02FFB0124DBE7184A64
:10125000184D136C43F000731364AA6D164B9A4239
:10126000D0D12B6E013B7E2BCCD8144A07CA01ABE0
:1012700083E807001846032100F08AFD6B6D834266
:101280004FF00003BED12A6D8A4201BFAB65054B0A
:101290002A6E1A7003BF0A4BEA6D1A601C46B2E749
:1012A0009AAD44C5E4240020D0560020160000204A
:1012B00000380240006600405041A0B0586600402F
:1012C0001023002037B500F095FD1D4D1D4C2881E1
:1012D000022321681C486B71012201F0A5FB1B4809
:1012E000216850F8D83F01225B689847002301939A
:1012F000174B184900931848184B4FF4805202F0CE
:1013000005F8174B197811B1134802F027F801F0CE
:1013100009FD0446FFF7C2FB4FF4C873B0FBF3F2BC
:1013200002FB130304F5167010FA83F00D4B1860DE
:1013300003F064FF08B10F232B8103B030BD00BF61
:10134000D824002010230020203500202045002034
:10135000D50D0008E8240020F0340020E50E000838
:10136000E4240020EC3400202DE9F04F2DED028B19
:10137000DFF8508293B00BAF9FED838BFFF7D0FC6B
:1013800000230A93ADF834300B937B600025844C26
:10139000DFF810A22E4601238DF81C3023688DED56
:1013A000008B4FF0000BD3F808908DF81DB05B4612
:1013B0000DF11D0207A92046C8479DF81C90B9F100
:1013C000000F24D0D8F8143083F48073C8F8143098
:1013D000102259460EA800F067FA236808AA5E6931
:1013E0000AA90DF11E032046B04797E803000FAB92
:1013F00083E803009DF834308DF844300A9B0E9347
:101400000EA9DDE90823504602F062FA4E4605F2C5
:10141000364540F66C0304F586549D4204F11804E9
:10142000B9D1002EB2D15F4801F0A0FF002840D111
:101430005D4D01F077FC2B6898423AD301F072FCC5
:101440000446FFF72BFB4FF4C873B0FBF3F202FB2B
:10145000130304F5167010FA83F02860534D8DF8CD
:1014600028602E7816B901238DF82830C6F11004B3
:10147000E4B20EA8FFF72AFB062C28BF06240EAB09
:10148000224699190DF1290000F0E8F90AAB0393FF
:10149000182302930134464B0193E4B201230093D5
:1014A000404804943AA3D3E9002301F0A5FF0023A8
:1014B0002B7001F037FC3F4A3F4C1368C31AB3F559
:1014C0007A7F2FD3106001F02FFC02460B4635487F
:1014D00002F02AF8334801F049FF18B3237A374D58
:1014E000002B14BF032302236B7101F01BFC0EAE13
:1014F0004FF47A730122B0FBF3F03146286028469E
:1015000000F0F8FA182302932D4B019380B240F2B9
:101510005513CDE90360009322481FA3D3E90023AC
:1015200001F06AFF237A93B101F0FCFB0025064627
:101530004FF48A7794F8D900284400F0030007FBA1
:10154000004393F8E82072B10135042DF2D1C82090
:1015500003F072F9237A002B7FF40DAF13B0BDECCA
:10156000028BBDE8F08FD3F8E02042B12368FA2B5C
:1015700038BFFA23B21A0533B2EB430FE4D3FFF7B7
:101580007FFB0028E0D1E2E700000000000000003F
:10159000401DA12026812A0BF1C6A7C1D068080FE3
:1015A00020350020F0340020EC340020E934002005
:1015B000E8340020005C0020D0560020D824002011
:1015C000045C00200008024008B5064800F08EFFC9
:1015D000054800F08BFFBDE80840044A044900209C
:1015E00004F076BF20350020F8450020445C002040
:1015F000A10E000870B50F4B1B780133DBB2012B35
:101600000C4611D80C4D29684FF47A730E6AA2FB70
:101610000332014622462846B047844204D1074B94
:1016200000221A70012070BD4FF4FA7003F004F923
:101630000020F8E71C230020B85E0020345C002066
:1016400007B50023024601210DF107008DF8073090
:10165000FFF7D0FF20B19DF8070003B05DF804FB51
:101660004FF0FF30F9E700000A4608B50421FFF704
:10167000C1FF80F00100C0B2404208BD30B4054C4B
:101680002368DD69044B0A46AC460146204630BC5F
:10169000604700BFB85E0020A086010070B503F06F
:1016A000FBFB094E094D30800024286833888342B3
:1016B00008D903F0EBFB2B6804440133B4F5803FF9
:1016C0002B60F2D370BD00BF365C0020085C0020A8
:1016D00003F092BC00F1006000F5803000687047B4
:1016E00000F10060920000F5803003F01BBC0000A8
:1016F000054B1A68054B1B889B1A834202D910447C
:1017000003F0C4BB00207047085C0020365C00205A
:10171000024B1B68184403F0C1BB00BF085C0020EB
:10172000024B1B68184403F0D1BB00BF085C0020CB
:1017300010F003030AD1B0F5047F05D200F1005088
:10174000A0F51040D0F80038184670470023FBE79A
:1017500000F10050A0F51040D0F8100A70470000CA
:10176000064991F8243033B10023086A81F8243007
:101770000822FFF7B5BF0120704700BF0C5C0020B6
:10178000014B1868704700BF002004E070B5194B8A
:101790001D68194B0138C5F30B0408442D0C0422B5
:1017A0001E88A6420BD15C680A46013C8242134661
:1017B0000FD214F9016F4EB102F8016BF6E7013A4E
:1017C00003F10803ECD181420B4602D22C2203F82C
:1017D000012B0A4A05241688AE4204D1984284BFE0
:1017E000967803F8016B013C02F10402F3D1581A18
:1017F00070BD00BF002004E0BC660008A8660008B9
:10180000022802BF024B4FF480729A61704700BFFA
:1018100000080240022802BF024B4FF080729A611A
:10182000704700BF00080240022801BF024A536906
:1018300083F48073536170470008024070B504461A
:101840004FF47A764CB1412C254628BF412506FB42
:1018500005F002F0F1FF641BF4E770BD10B5002342
:10186000934203D0CC5CC4540133F9E710BD0000AF
:1018700010B5013810F9013F3BB191F900409C428D
:1018800003D11AB10131013AF4E71AB191F90020FC
:10189000981A10BD1046FCE703460246D01A12F90A
:1018A000011B0029FAD1704702440346934202D03B
:1018B00003F8011BFAE770472DE9F8431F4D144662
:1018C00095F824200746884652BBDFF870909CB3F9
:1018D00095F824302BB92022FF2148462F62FFF7CC
:1018E000E3FF95F82400C0F10802A24228BF224677
:1018F000D6B24146920005EB8000FFF7AFFF95F8A6
:101900002430A41B1E44F6B2082E17449044E4B2BF
:1019100085F82460DBD1FFF723FF0028D7D108E04A
:101920002B6A03EB82038342CFD0FFF719FF002815
:10193000CBD10020BDE8F8830120FBE70C5C002040
:10194000024B1A78024B1A70704700BF345C0020BB
:101950001C23002010B5104C104802F0C3FA214699
:101960000E4802F0EBFA2468626DD2F8043843F0B6
:101970000203C2F804384FF47A70FFF75FFF08499A
:10198000204602F0E1FB626DD2F8043823F0020336
:10199000C2F8043810BD00BF14680008B85E00200B
:1019A0001C680008704700002DE9F0470D4604460A
:1019B00000219046284640F27912FFF775FF234632
:1019C00020220021284601F025FF231D022220218C
:1019D000284601F01FFF631D03222221284601F043
:1019E00019FFA31D03222521284601F013FF04F14E
:1019F000080310222821284601F00CFF04F11003EF
:101A000008223821284601F005FF04F111030822BD
:101A10004021284601F0FEFE04F11203082248216D
:101A2000284601F0F7FE04F1140320225021284635
:101A300001F0F0FE04F1180340227021284601F065
:101A4000E9FE04F120030822B021284601F0E2FE5D
:101A500004F121030822B821284601F0DBFE04F13D
:101A60002207C0263B46314608222846083601F0A8
:101A7000D1FEB6F5A07F07F10107F3D104F13203DF
:101A800008223146284601F0C5FE002704F1330A3A
:101A900094F832304FEAC7099F4209F5A47615D36E
:101AA000B8F1000F08D1314604F599730722284692
:101AB00001F0B0FE09F24F16274694F832213B1B85
:101AC00093420CD3F01DC008BDE8F0870AEB070372
:101AD00008223146284601F09DFE0137D8E707F27B
:101AE000331331460822284601F094FE08360137A8
:101AF000E3E7000013B504460846002101602346D1
:101B0000C0F803102022019001F084FE0198231DEB
:101B10000222202101F07EFE0198631D0322222172
:101B200001F078FE0198A31D0322252101F072FE29
:101B3000019804F108031022282101F06BFE072010
:101B400002B010BDF7B50023047F00910E460722B6
:101B50001946054601F022FD731C00930122002363
:101B60000721284601F01AFDC4B9B31C00930522D1
:101B700023460821284601F011FD0D243746B2788E
:101B8000BB1B934211D32B7FA88A0734E408BBB94F
:101B9000844294BF0020012003B0F0BDAB8ADB007B
:101BA000083BDB08B3700824E8E7FB1C00932146E0
:101BB00000230822284601F0F1FC08340137DEE753
:101BC000201A18BF0120E7E7F7B50023047F009132
:101BD0000E4608221946054601F0E0FC731CC4B904
:101BE0000822009311462346284601F0D7FC102412
:101BF000012372785F1C013B934211D32B7FA88A8B
:101C00000734E408BBB9844294BF0020012003B02C
:101C1000F0BDAB8ADB00083BDB0873700824E7E704
:101C2000F3190093214600230822284601F0B6FC50
:101C300008343B46DDE7201A18BF0120E7E7000023
:101C4000F8B50E4605461446002181223046FFF7BE
:101C50002BFE2B4608220021304601F0DBFD7CB92B
:101C60006B1C07220821304601F0D4FD0F2401230C
:101C70006A785F1C013B934204D3E01DC008F8BDA5
:101C80000824F4E7EB1921460822304601F0C2FD92
:101C900008343B46ECE70000F8B50E46054614460E
:101CA0000021CE223046FFF7FFFD2B4628220021DF
:101CB000304601F0AFFD7CB905F108030822282168
:101CC000304601F0A7FD30242F462A7A7B1B934231
:101CD00004D3E01DC008F8BD2824F5E707F1090387
:101CE00021460822304601F095FD08340137ECE723
:101CF000F7B5047F00910E4601231022002105460E
:101D000001F04CFCC4B9B31C0093092223461021F6
:101D1000284601F043FC192437467288BB1B9A42BF
:101D200011D82B7FA88A0734E408BBB9844294BF3A
:101D30000020012003B0F0BDAB8ADB00103BDB08C4
:101D400073801024E8E73B1D0093214600230822FE
:101D5000284601F023FC08340137DEE7201A18BFBB
:101D60000120E7E730B5094D0A4491420DD011F842
:101D7000013B5840082340F30004013B2C4013F082
:101D8000FF0384EA5000F6D1EFE730BD2083B8EDC1
:101D9000F7B54FF0FF33DFF854C0DFF854E000EB45
:101DA00081011A4688421CD050F8044B019401AFBF
:101DB000042417F8015B82EA05620825DB18164641
:101DC00005F1FF355241002EBCBF83EA0C0382EAC5
:101DD0000E0215F0FF05F1D1013C14F0FF04E8D12B
:101DE000E0E7D843D14303B0F0BD00BF9336EAA982
:101DF000EBE1F042F7B5384A106851686B4603C30F
:101E00006A4636493648082304F0C2FB04460028D7
:101E100033D10A25334A106851686B4603C36A46BA
:101E200031492F48082304F0B3FB0446002849D069
:101E30000369B3F5E02F45D8B0F8661041F270722F
:101E400091423FD1294A024402F15C018B4239D3CD
:101E50005C3B234900209E1AFFF784FF3246074669
:101E600004F164010020FFF77DFFA3689F4229D1A0
:101E7000E368984208BF002524E00369B3F5E02F2A
:101E800027D8418B41F27072914220D1174A024407
:101E900002F110018B4218D3103B114900209D1A0A
:101EA000FFF760FF2A46064604F118010020FFF7FD
:101EB00059FFA3689E4202D1E368984201D00D25E4
:101EC000A8E70025284603B0F0BD1025A2E70C25A1
:101ED000A0E70B259EE700BFDC660008DCFF0600DC
:101EE00000000108E566000890FF06000800FFF703
:101EF00010B5037C044613B9006804F031FB20469A
:101F000010BD00000023BFF35B8FC360BFF35B8F86
:101F1000BFF35B8F8360BFF35B8F7047BFF35B8F53
:101F20000068BFF35B8F704770B505460C30FFF754
:101F3000F5FF05F1080604463046FFF7EFFFA04223
:101F400006D930466D68FFF7E9FF2544281A70BDB1
:101F50003046FFF7E3FF201AF9E7000070B50546A9
:101F6000406898B105F10800FFF7D8FF05F10C06AD
:101F700004463046FFF7D2FF8442304694BF6D6876
:101F80000025FFF7CBFF013C2C44201A70BD000058
:101F900038B50C460546FFF7C7FFA04210D305F140
:101FA0000800FFF7BBFF04446868B4FBF0F100FBD6
:101FB0001144BFF35B8F0120AC60BFF35B8F38BD72
:101FC0000020FCE72DE9F041144607460D46FFF7D7
:101FD000C5FF844228BF0446D4B1B84658F80C6BFC
:101FE0004046FFF79BFF3044286040467E68FFF77D
:101FF00095FF331A9C4203D86C600120BDE8F08144
:102000006B60A41B3B68AB602044E8600220F5E7EE
:102010002046F3E738B50C460546FFF79FFFA04280
:1020200010D305F10C00FFF779FF04446868B4FB96
:10203000F0F100FB1144BFF35B8F0120EC60BFF3B4
:102040005B8F38BD0020FCE72DE9FF4188466946DB
:102050000746FFF7B7FF6C4606B204EBC60600253D
:10206000B44209D06268206808EB0501FFF7F6FB6F
:10207000636808341D44F3E729463846FFF7CAFF72
:10208000284604B0BDE8F081F8B505460C300F468F
:10209000FFF744FF05F1080604463046FFF73EFF10
:1020A000A042304688BF6C68FFF738FF201A3860BE
:1020B00020B130462C68FFF731FF2044F8BD000006
:1020C00073B5144606460D46FFF72EFF844228BF1F
:1020D00004460190DCB101A93046FFF7D5FF019B12
:1020E00033B93268C5E90233C5E9002401200CE0A8
:1020F0009C4238BF01942860019868608442F5D9F9
:102100003368AB60241AEC60022002B070BD204638
:10211000FBE700002DE9FF410F466946FFF7D0FFBE
:102120006C4600B204EBC0050026AC4209D0D4F8DE
:10213000048054F8081BB8194246FFF78FFB464449
:10214000F3E7304604B0BDE8F081000038B505463D
:10215000FFF7E0FF044601462846FFF719FF204637
:1021600038BD000010B4026854681A4623465DF872
:10217000044B18470020704700207047704700004C
:10218000002070470E20704700F5805090F8C8007E
:10219000C0F340007047000000F5805090F9D00077
:1021A0007047000000F58050C0F8CC100120704747
:1021B000F7B50C68BDF8207014F0005470D10D7B99
:1021C000082D6DD8302585F311884569AE687601F4
:1021D0000CD4AC68240108D4AC6814F080545DD1F0
:1021E00084F31188204603B0F0BD01240E6804F189
:1021F000180C002EB8BFF6004FEA0C1CB4BF46F016
:102200000406760545F80C600E680FFA84FC16F09B
:10221000804F18BF05EB0C1E05EB0C1C1EBFDEF833
:10222000806146F00206CEF880610E7BCCF88461B6
:1022300005EB04158E68C5F88C614E68C5F8886199
:10224000DCF8805145F00105CCF8805100EB4416D4
:1022500041F268052E4405EB44150544C6E9002308
:1022600008350E4601F10C0C56F804EB45F804EB6A
:102270006645F9D1843436882E8000EB441407F08B
:102280000305267926F00B0635432571002484F3D7
:102290001188009700F068FD0120A4E70224A5E75B
:1022A0004FF0FF309FE7000013B500F58054019117
:1022B000E06DFFF753FE1F280AD90199E06D202237
:1022C000FFF7C2FEA0F120035842584102B010BDF2
:1022D0000020FBE708B5302383F3118800F5805018
:1022E000C06DFFF70FFE002383F3118808BD0000C7
:1022F00000220260828142608260704710B5002235
:102300000023C0E900230023044603810C30FFF7BB
:10231000EFFF204610BD0000F0B5054600F58050E7
:102320000C4690F8C83013F0040FC3F3800108BFC7
:10233000114661F3820304F1840680F8C83005EB8E
:10234000461389B01B79D8072ED57AB319072DD437
:102350006846FFF7D3FF05EB441303F5835303F1FE
:10236000180703AA103318685968144603C40833C1
:10237000BB422246F7D1186820609B88A380DDE924
:102380000E23CDE900230123ADF808302B68694600
:10239000DB6B2846984705EB46152B791A075CBF7F
:1023A00043F008032B7101E0002AF4D109B0F0BD1D
:1023B0002DE9F0479A4688B0074688469146302373
:1023C00083F3118807F580546846FFF797FFE06DA7
:1023D000FFF7AAFD1F282AD9E06D20226946FFF7E2
:1023E000B5FE202823D103AD444605AB2E4603CECF
:1023F0009E4220606160354604F10804F6D13068E1
:102400002060B388A380DDE90023C9E90023BDF87B
:102410000830AAF80030002383F3118853464A4657
:102420004146384608B0BDE8F04700F08BBC0020BC
:1024300080F3118808B0BDE8F08700002DE9F84F5F
:102440000023C0E90133264B044640F8183B0F46F1
:10245000FFF74EFF04F12800FFF750FF04F1480892
:1024600004F582554646083530462036FFF746FFCC
:10247000AE42F9D104F580554FF480534FF0000976
:10248000C5E91339C5F848800123EE6504F587587E
:1024900004F58456C5F8549085F8583085F86030B6
:1024A000083608F108084FF0000A4FF0000B46E923
:1024B00008ABA6F11800FFF71BFF203646F8289C52
:1024C0004645F4D1012F85F8D07002D9054800F0B7
:1024D00023FC054B53F8273063612046BDE8F88F95
:1024E00028670008F06600080C67000810B5044B68
:1024F000197804464A1C1A70FFF7A0FF204610BD49
:10250000405C00202DE9F047002950D0294B2A4F8C
:10251000B7FBF1F599428CBF0A231123581EB5FB76
:10252000F3FC03FB1C53C4B22BB102280346F5D8BD
:102530000020BDE8F0870CF1FF36B6F5806FF7D2CA
:10254000C4EBC40E0EF103034FEAE309C3F3C70360
:10255000A4EB030809F1010A4FF47A755FFA88F0D9
:1025600009FB05555AFA88F8B5FBF8F5B5F5617F12
:10257000C1BF0EF1FF33C3F3C703E01AC0B25C1C46
:1025800050FA84F40CFB04F4B7FBF4F4A142CFD16D
:10259000013BDBB20F2BCBD80138C0B20728C7D81C
:1025A0000021107116809170D3700120C1E7084698
:1025B000BFE700BF3F420F0080DE800270B50546D6
:1025C0000E464FF47A746B695B6803F00103B34203
:1025D00007D04FF47A7002F02FF9013CF3D1204676
:1025E00070BD0120FCE7000030B54269936913F02B
:1025F000700F16D000230B4C936103F1840200EBA3
:10260000421211794D0709D5890707D5416954F858
:1026100023508D60117941F0040111710133032BB6
:10262000EBD130BD1467000873B51D4643691646EB
:102630009A68D207044609D59A6801219960C2F3C5
:102640004002CDE900650021FFF766FE63699A68E4
:10265000D1050BD59A684FF480719960C2F340227E
:10266000CDE9006501212046FFF756FE63699A68AF
:10267000D2030BD59A684FF480319960C2F340427F
:10268000CDE9006502212046FFF746FE04F58053A0
:10269000D3F8CC0010B103681B699847204602B0FC
:1026A000BDE87040FFF7A0BF0C4B10B51C561B5C7B
:1026B000012B11D800F038FB50EA0103024602D08A
:1026C000421E61F10001064B53F8240020B1BDE821
:1026D00010400B46FFF7A8BF10BD00BF08670008F9
:1026E000385C0020F8B504464669002972D106F12D
:1026F0000C073868800770D006EB01153868D5F8EC
:10270000B00110F0040FD5F8B0011ABFC00840F0B6
:102710000040400DA061D5F8B0C11CF0020F1CBFF5
:1027200040F08040A061D5F8B40106EB011100F043
:102730000F0084F82400D1F8B8012077D1F8B8014F
:10274000000A6077D1F8B801000CA077D1F8B80181
:10275000000EE077D1F8BC0184F82000D1F8BC016C
:10276000000A84F82100D1F8BC01000C84F8220092
:10277000D1F8BC11090E84F823103821396004F116
:10278000340004F1180104F1240551F8046B40F8F9
:10279000046BA942F9D109880180C4E90A232146C2
:1027A0000023238651F8283B2046DB6B984704F52D
:1027B000805393F8C820D3F8CC0042F0040283F889
:1027C000C82010B103681B6998472046BDE8F8404F
:1027D000FFF70ABF06F110078BE7F8BD0D4B70B588
:1027E0001D561B5C012B0C4612D800F09DFA0246C8
:1027F0000B4652EA030102D0013A63F10003064995
:1028000051F8250020B12146BDE87040FFF76ABFAE
:1028100070BD00BF08670008385C0020F0B53021AB
:1028200081F31188DFF848C000F583510831002496
:1028300004F1840500EB45152E7977070ED4F606D2
:102840000CD5D1E9007697429E4107D246695CF8E3
:102850002470B7602E7946F004062E710134032CE3
:1028600001F12001E4D1002383F31188F0BD00BF02
:102870001467000808B5302383F31188FFF7B4FE0E
:10288000002383F3118808BDF8B5436905469868AD
:1028900000F0E050B0F1E05F0F4621D0F8B13023F6
:1028A00083F3118805F583541034002606F1840360
:1028B00005EB43131B791A0706D50136032E04F1E5
:1028C0002004F3D1012007E05B07F6D42146384607
:1028D00000F084FA0028F0D1002383F31188F8BDBA
:1028E0000120FCE708B5302383F3118800F5805000
:1028F000C06DFFF719FB002383F3118843090CBF58
:102900000120002008BD0000F8B51D46002313700B
:102910000F4606461446FFF7E5FF80F001003870C9
:1029200025B129463046FFF7AFFF2070F8BD000003
:102930002DE9B8410C4615461F46804600F0F4F9D3
:102940000B462178024609B9287850B14046FFF776
:1029500065FFFFF78FFF3B462A462146FFF7D4FF6E
:102960000120BDE8B881000038B5302383F3118819
:1029700000F580542A4D94F8D030EB5CE3B1012B84
:1029800028D0002383F3118894F8C830DB0712D4D1
:1029900089B1302383F3118894F8D030EB5C33B3E2
:1029A000012B31D094F8C83043F0010384F8C830CB
:1029B000002383F3118838BD1A4B1A6C42F0007261
:1029C0001A641A6A42F000721A621A6A22F00072DD
:1029D0001A62D6E7134B1A6C42F080621A641A6AC4
:1029E00042F080621A621A6A22F08062F0E70321E4
:1029F000132001F0E7F90321142001F0E3F903218A
:102A0000152001F0DFF9CDE703213F2001F0DAF9CD
:102A10000321402001F0D6F903214120F1E700BF56
:102A200004670008003802402DE9F04700F58055A2
:102A300088B095F8D030022B04468846164600F23E
:102A40008180854F57F823200AB947F82300D7F82B
:102A500000A0C4F80C802674BAF1000F64D095F879
:102A6000D030012B70D001212046FFF77DFF3023AD
:102A700083F311886269136823F0020313606269AB
:102A8000136843F001031360636900275F6187F3F4
:102A9000118801212046FFF791FD002800F0958064
:102AA000E86DFFF72FFA04F58359BA4609F10809D2
:102AB000202200216846FEF7F7FE02A8FFF718FC67
:102AC000CDF818A06A4609EB07030DF1180E9446DD
:102AD000BCE80300F44518605960624603F108033E
:102AE000F5D1DCF80000186020379CF804201A713A
:102AF000602FDDD195F8C8306FF38203002785F889
:102B0000C8306A4641462046ADF80070ADF8027004
:102B10008DF80470FFF7F6FC636948BB4FF4004280
:102B20001A6008B0BDE8F08741F2D80003F0D8FC85
:102B3000814610B15146FFF781FCC7F80090B9F10A
:102B4000000F8CD10020ECE7386803681B6B9847B6
:102B50000146002887D13868FFF706FF3868036808
:102B600032465B684146984700287FF47CAFE9E72E
:102B700061221A609DF802309DF803201B061204A2
:102B800002F4702203F040731343BDF80020C2F337
:102B9000090213439DF804201205022E02F4E002FC
:102BA0000CBF4FF000410021134362690B43D36116
:102BB000636913225A616269136823F00103136089
:102BC00039462046FFF7FAFC08B96369A6E795F88D
:102BD000D030002B39D16169D1F8002242F00102D6
:102BE000C1F800226169D1F8002222F47C5222F05F
:102BF0000E02C1F800226169D1F8002242F460623D
:102C0000C1F800226269C2F814326269C2F8043263
:102C100062696FF07841C2F80C126269C2F8403202
:102C20006269C2F844326269C2F8B0326269C2F8BD
:102C3000B432636944F20102C3F81C226269D2F81B
:102C4000003223F00103C2F8003295F8C83043F097
:102C5000020385F8C83064E7385C002008B500201E
:102C6000FFF722FDBDE8084001F082B808B5002159
:102C70000846FFF7B3FDBDE8084001F079B8000051
:102C800008B501210020FFF7A9FDBDE8084001F0CB
:102C90006FB8000008B50120FFF706FDBDE8084049
:102CA00001F066B808B500210120FFF797FDBDE8E7
:102CB000084001F05DB8000008B501210846FFF7A3
:102CC0008DFDBDE8084001F053B8000000B59BB091
:102CD000EFF3098168226846FEF7C0FDEFF3058334
:102CE000014B9B6BFEE700BF00ED00E008B5FFF76E
:102CF000EDFF000000B59BB0EFF309816822684644
:102D0000FEF7ACFDEFF30583014B5B6BFEE700BF05
:102D100000ED00E0FEE700000FB408B5029801F0F6
:102D200031FDFEE702F0B6B902F098B913B56C4672
:102D300084E80600031D94E8030083E805000120F1
:102D400002B010BD73B58568019155B11B885B0752
:102D500007D4D0E900369B6B9847019AC1B2304640
:102D6000A847012002B070BDF0B5866889B005465D
:102D70000C465EB1BDF838305B070AD4D0E90037A5
:102D80009B6B98472246C1B23846B047012009B034
:102D9000F0BD00220023CDE900230023ADF8083068
:102DA0000A4603AB01F10806106851681C4603C4CB
:102DB0000832B2422346F7D1106820609288A28080
:102DC000FFF7B2FF0423ADF808302B68CDE900010E
:102DD000DB6B694628469847D8E7000030B50368A2
:102DE0000968DD0FB5EBD17F23F0604421F060422C
:102DF0004FEAD1700BD0002BB8BFA40C0029B8BF8C
:102E0000920C944202D034BF0120002030BD944285
:102E100005D1C1F38070C3F380738342F6D194422D
:102E20002CBF00200120F1E72DE9F041456A15B9DA
:102E30004162BDE8F0814B6823F06047C3F38A46E6
:102E40004FEAD37EC3F3807816EA230638BF3E46A6
:102E5000AC462B465A68BEEBD27F22F060440AD0C3
:102E6000002A18DAA40CB44217D19D420FD10D608C
:102E7000DEE71346EEE7A74207D102F08044C2F333
:102E8000807242450BD054B1EFE708D2EDE7CCF8A1
:102E900000100B60CDE7B44201D0B442E5D81A6807
:102EA0009C46002AE5D11960C3E700002DE9F047F0
:102EB000089D01F007044FEAD508224405F00705F4
:102EC00000EBD1004FF47F49944201D1BDE8F08777
:102ED00004F0070705F0070A57453E4638BF564637
:102EE000C6F10806111B8E4228BF0E46E10808EB0A
:102EF000D50E415C13F80EC0B94029FA06F721FA45
:102F00000AF1FFB28CEA010147FA0AF739408CEA6C
:102F1000010C03F80EC034443544D5E780EA0120A3
:102F2000082341F2210201B24000002980B203F1DE
:102F3000FF33B8BF504013F0FF03F4D170470000D7
:102F400038B50C468D18A54200D138BD14F8011BC8
:102F5000FFF7E4FFF7E7000042684AB113684360F7
:102F60004389818901339BB29942438138BF838170
:102F70001046704770B588B0202204460D4668465A
:102F80000021FEF791FC20460495FFF7E5FF02467D
:102F900058B16B46054608AE1C4603CCB4422860C7
:102FA0006960234605F10805F6D1104608B070BDEA
:102FB000082817D909280CD00A280CD00B280CD0C7
:102FC0000C280CD00D280CD00E2814BF4020302027
:102FD00070470C207047102070471420704718204D
:102FE0007047202070470000082817D90C280CD9FA
:102FF00010280CD914280CD918280CD920280CD941
:1030000030288CBF0F200E207047092070470A20FF
:1030100070470B2070470C2070470D207047000050
:103020002DE9F843078C072F04461ED9D0E90298F2
:1030300000254FF6FF73C5F12006A5F1200029FAFF
:1030400005F108FA06F628FA00F031430143C9B247
:103050001846FFF763FF0835402D0346EBD1E169C1
:103060003A46BDE8F843FFF76BBF4FF6FF70BDE887
:10307000F883000010B54B6823B9CA8A63F30902CC
:10308000CA8210BD04691A681C600361C38A013BCF
:10309000C3824A60EFE700002DE9F84F1D46CB8A56
:1030A0000F46C3F309010529814692460B4630D0ED
:1030B0000020AAB207F11A049EB2042E1FFA80F86B
:1030C0000FD8904503F1010306D3FB8A0A4462F34B
:1030D0000903FB8201201AE01AF80060E65401306F
:1030E000EAE79045F1D2A1F1050B1C237C68BBFBFC
:1030F000F3F203FB12BB1FFA8BF6002C45D14846B6
:10310000FFF72AFF044638B978606FF00200BDE887
:10311000F88F4FF00008E6E7002606607860ADB251
:103120004FF0000B454510D90AEB0803221D13F898
:10313000011B9155B1B208F101081B291FFA88F84B
:103140002BD0454506F10106F1D8FB8AC3F30902ED
:10315000154465F30903BCE7013292B21C462368AB
:10316000002BF9D16B1F0B441C21B3FBF1F301338E
:103170009BB29A42D3D2BBF1000FD0D14846FFF7A1
:10318000EBFE20B9C4F800B0BFE70122E7E7C0F8C2
:1031900000B05E4620600446C1E74545D5D94846A3
:1031A000FFF7DAFE08B92060AFE7C0F800B00026EC
:1031B00020600446B6E700002DE9F04F2DED028BAC
:1031C0001C4683B05B69019207468846002B00F0DD
:1031D0009A80238C2BB1E269002A00F09480072B9F
:1031E00035D807F10C00FFF7B7FE054638B96FF088
:1031F0000205284603B0BDEC028BBDE8F08F142217
:103200000021FEF751FB228CE16905F10800FEF771
:1032100025FB208C013080B2FFF7E6FEFFF7C8FEE9
:10322000013880B22084013028746369228C1B78B5
:103230002A4403F01F0363F03F0348F00041137278
:10324000384669602946FFF7EFFD0125D1E700F117
:103250000C034FF0000908EE103A4FF0800A4E467A
:103260004D4618EE100AFFF777FE83460028BED0C1
:1032700014220021FEF718FB002E3AD1019BABF877
:10328000083002220BF1080E1FFA82FC0CF101003B
:10329000BCF1060F218C80B201D88E422BD3FFF7F0
:1032A000A3FEFFF785FE62691278013802F01F0263
:1032B0008E4208BF4FF0400A42EA49121BFA80F1E1
:1032C0004AEA020A013048F0004281F808A08BF86F
:1032D0001000CBF8042059463846FFF7A5FD238C93
:1032E0000135B3422DB289F001094FF0000AB8D17F
:1032F0007FE70022C6E7E169895D0EF8021001361A
:10330000B6B20132C0E76FF0010572E7F8B51546B5
:103310000E463022002104461F46FEF7C5FA069BE2
:103320006360B5F5001F079BA76034BF6A094FF6BD
:10333000FF72A36297B2E66104F1100000239A4283
:1033400006D800230360A782E3822383E360F8BDED
:103350000660013330462036F1E7000003781BB9E0
:103360004BB2002BC8BF0170704700000078704757
:10337000F8B50C46C969074611B9238C002B37D123
:10338000257E1F2D34D8387828BB228C072A2CD8CC
:10339000268A36F003032BD14FF6FF70FFF7D0FDDE
:1033A00020F001003102400441EA0561400C41EA8D
:1033B00040254FF6FF72234629463846FFF7FCFEAC
:1033C000002807DD626913780133DBB21F2B88BF49
:1033D00000231370F8BD218A2D0645EA0125054317
:1033E0002046FFF71DFE0246E5E76FF00300F1E718
:1033F0006FF00100EEE7000070B58AB00446164693
:103400000021282268461D46FEF74EFABDF83830E6
:10341000ADF810300F9B05939DF840308DF81830B3
:10342000119B07936946BDF84830ADF8203020461F
:10343000CDE90265FFF79CFF0AB070BD2DE9F041B0
:10344000D36905460C4616460BB9138C5BBB377E19
:103450001F2F28D895F80080B8F1000F26D03046ED
:10346000FFF7DEFD3378210241EAC33141EA08016A
:10347000338A41EA076141EA03410246334641F09B
:1034800080012846FFF798FE00280ADD3378012BDB
:1034900007D1726913780133DBB21F2B88BF002379
:1034A0001370BDE8F0816FF00100FAE76FF00300E0
:1034B000F7E70000F0B58BB004460D461746002133
:1034C000282268461E46FEF7EFF99DF84C305A1E3A
:1034D000534253418DF800309DF84030ADF8103024
:1034E000119B05939DF848308DF81830149B079375
:1034F0006A46BDF85430ADF8203029462046CDE963
:103500000276FFF79BFF0BB0F0BD0000406A00B1F0
:1035100004307047436A1A68426202691A600361A4
:10352000C38A013BC38270472DE9F041D0F8208067
:10353000194E14461D464146002709B9BDE8F081E1
:10354000D1E90223A21A65EB0303964277EB03034A
:103550001ED2036A8B420DD1FFF78CFD036A1B68F4
:10356000036203690B60C38A0161016A013BC38284
:103570008846E2E7FFF77EFD0B68C8F80030036974
:103580000B60C38A0161013BC382D8F80010D4E705
:1035900088460968D1E700BF80841E002DE9F04FFE
:1035A0008BB00D46DDF8509014469B4680460028AF
:1035B00000F01981B9F1000F00F01581531E3F2B67
:1035C00000F21181012A03D1BBF1000F40F00B8101
:1035D0000023CDE90833B8F81430B5EBC30F4FEA38
:1035E000C30703D300200BB0BDE8F08F2B199F4217
:1035F000D8F80C303ABF7F1BFFB227461BB9D8F86A
:103600001030002B7AD0272D4ED8C5F12806B742AE
:103610004FF000032CBFF6B23E4600932946D8F87F
:10362000080008AB3246FFF741FCA7EB060A354419
:103630005FFA8AFAB8F8143003F10053053BDB0057
:103640000493D8F80C3003932821039B13B1BAF1EB
:10365000000F2CD1D8F8100040B1BAF1000F05D0FE
:10366000009608AB5246691AFFF720FC38B2002FCB
:10367000B8D066070AD00AAB03EBD401624211F856
:10368000083C02F00702134101F8083C082C3CD921
:10369000102C40F2B580202C40F2B780BBF1000F17
:1036A00000F09C80082334E0BA460026C2E7049B61
:1036B000E02B28BFE02306930B44AB42059314D9BB
:1036C0005A1B03980096924534BF5246D2B2691AEB
:1036D00008AB04300792FFF7E9FB079A1644AAEB00
:1036E000020A1544F6B25FFA8AFA049B069A059913
:1036F0009B1A0493039B1B680393A6E70093D8F8D7
:10370000080008AB3A462946AEE7BBF1000F13D0DC
:103710000123B4EBC30F6CD0082C12D89DF82030D5
:10372000621E23FA02F2D50706D54FF0FF3202FAE5
:1037300004F423438DF820309DF8203089F80030C0
:1037400051E7102C12D8BDF82030621E23FA02F285
:10375000D10706D54FF0FF3202FA04F42343ADF847
:103760002030BDF82030A9F800303CE7202C0FD8DD
:103770000899631E21FA03F3DA0705D54FF0FF32EB
:1037800002FA04F40C430894089BC9F800302AE7B5
:10379000402C2BD0DDE90865611EC4F12102A4F1A3
:1037A000210326FA01F105FA02F225FA03F3114387
:1037B0001943CB0712D50122A4F12003C4F1200143
:1037C00002FA03F322FA01F1A240524243EA010352
:1037D00063EB430332432B43CDE90823DDE90823A0
:1037E000C9E90023FFE66FF00100FCE66FF0080076
:1037F000F9E6082CA0D9102CB3D9202CEED8C3E7B9
:10380000BBF1000FADD0022383E7BBF1000FBBD0AB
:1038100004237EE730B5012A144638BF0124402C2A
:1038200085B028BF40240025012ACDE9025518D8CB
:103830001B788DF8083063070AD004AB03EBD4057E
:10384000624215F8083C02F00702934005F8083C74
:10385000009103462246002102A8FFF727FB05B08E
:1038600030BD082AE4D9102A03D81B88ADF80830E7
:10387000E1E7202A8DBFD3E900231B680293CDE93D
:103880000223D8E710B5CB681BB98B600B618B8224
:1038900010BD04691A681C600361C38A013BC382BE
:1038A000CA60F0E703064CBFC0F3C0300220704787
:1038B00008B50246FFF7F6FF022806D15306C2F309
:1038C0000F2001D100F0030008BDC2F30740FBE761
:1038D0002DE9F04F93B0CDE903230A680446104662
:1038E000FFF7E0FF022814BFC2F306260026002AD5
:1038F0000D46824680F2F28112F0C04940F0EE811E
:10390000097B002900F0EA81022803D02378B34222
:1039100040F0E781C2F304630693104602F07F0390
:103920000593FFF7C5FF059B29444FEA834848EA02
:103930000A4848EA4668CE7800230022CDE90823E9
:10394000F309834648EA0008029367D0059B009379
:1039500002466768534608A92046B847002800F089
:10396000C381276A4FB9414604F10C00FFF702FBFF
:10397000074690B96FF0020054E03B6998450DD0BE
:103980003F68002FF9D1414604F10C00FFF7F2FA2D
:1039900007460028EED0236A3B60276297F817C0DD
:1039A00006F01F08CCF3840CACEB08001FFA80FE75
:1039B0000028B8BF0EF12000A8EB0C031FFA83FE0D
:1039C000D7E90221B8BF00B2002B0793BEBF0EF1AA
:1039D00020031BB2079352EA010338D0039BDFF8A0
:1039E00024E39A1A049B4FF0000C63EB0101964507
:1039F0007CEB01032BD36B7B97F81AE0734519D14D
:103A0000029B002B78D0012821DC7868F8B9DFF818
:103A1000F0C2944570EB010316D337E0276A27B94B
:103A20006FF00C0013B0BDE8F08F3B699845B5D03E
:103A30003F68F4E7B24890427CEB010301D30020D9
:103A4000F0E7029B002BFAD0079B0F2B17DCFA7DC7
:103A5000B30002F0030203F07C031343FB75394605
:103A60002046FFF707FB6B7BBB76029B3BB9FB7DD8
:103A7000C3F38402013262F38603FB75D0E76A7BED
:103A8000BB7E9A42DBD1029B002B35D0B309022BBF
:103A900032D0039BBB60049BFB60142200210DA865
:103AA000FDF702FF039B0A93049B0B932B1D0C93C2
:103AB0002B7BADF83EB0013BDBB2ADF83C30069B52
:103AC0008DF84230059B8DF8433094F82C308DF8FA
:103AD00040A083F001038DF844308DF84180A36845
:103AE0000AA920469847FB7DC3F38403013303F002
:103AF0001F039B02FB82A2E7FB7DC6F34012B2EBE1
:103B0000D31F40F0F480C3F38403434540F0F280B8
:103B1000029A2B7BB609002A4DD0F2075DD4032B05
:103B200040F2EB80039BBB60049BFB602B7BAE1DD4
:103B3000033BDBB23246394604F10C00FFF7ACFA26
:103B400000280CDA39462046FFF794FAFB7DC3F3D0
:103B50008403013303F01F039B02FB820AE7DDE9C4
:103B60000884AB883B834FF6FF73C9F12000A9F1AD
:103B7000200228FA09F104FA00F0014324FA02F2C3
:103B800011431846C9B2FFF7C9F909F10809B9F19B
:103B9000400F0346E9D1B8822A7B033AD2B23146BC
:103BA000FFF7CEF9FB7DB882DA43C2F3C01262F3AD
:103BB000C713FB7543E786B92E1D013BDBB23246C6
:103BC000394604F10C00FFF767FA0028BADB2A7BBC
:103BD000B88A013AD2B23146E2E7F98AC1F3090163
:103BE000013B0429DAB25BD8281D002307F11B062C
:103BF0009A4208D910F801CB06F801C0013101330F
:103C00000529DBB2F4D103990A9104990B919342EF
:103C100007F11B010C9138BF043379680D9134BF53
:103C200055FA83F300230E93FB8AADF83EB0C3F33D
:103C300009031A44069B8DF84230059B8DF84330EA
:103C400094F82C30ADF83C2083F001038DF844301B
:103C500000238DF840A08DF841807B602A7BB88AD4
:103C6000013A291DFFF76CF93B8BB882834203D1DF
:103C7000A3680AA92046984720460AA9FFF702FE32
:103C8000FB7DBA8AC3F38403013303F01F039B0255
:103C9000FB823B8B9A420CBF00206FF01000C1E604
:103CA0007B68002BAFD0052001E01C3033461E6836
:103CB000002EFAD1091A081D2E1D184401EB090C1B
:103CC000BCF11B0F5FFA89F39DD89A429BD916F875
:103CD000013B00F8013B09F10109EFE76FF0090032
:103CE000A0E66FF00A009DE66FF00B009AE66FF019
:103CF0000D0097E66FF00E0094E66FF00F0091E66E
:103D000040420F0080841E00EFF3098305494A6B8F
:103D100022F001024A63683383F30988002383F3A6
:103D20001188704700EF00E0302080F3118862B600
:103D30000C4B0D4AD96821F4E0610904090C0A43CF
:103D4000DA60D3F8FC20094942F08072C3F8FC2005
:103D50000A6842F001020A602022DA7783F8220022
:103D6000704700BF00ED00E00003FA05001000E01E
:103D700010B5302383F311880E4B5B6813F4006396
:103D800014D0F1EE103AEFF30984683C4FF08073E1
:103D9000E361094BDB6B236684F3098800F0BCFC0C
:103DA00010B1064BA36110BD054BFBE783F31188EF
:103DB000F9E700BF00ED00E000EF00E03F0300087E
:103DC0004203000800F1604303F561430901C9B2F1
:103DD00083F80013012200F01F039A4043099B005F
:103DE00003F1604303F56143C3F880211A60704713
:103DF000026843681143016003B11847704700002F
:103E000013B5446BD4F894341A681178042915D189
:103E1000217C022912D11979128901238B40134286
:103E20000CD101A904F14C0001F09EFFD4F8944498
:103E3000019B21790246206800F0D0F902B010BD44
:103E4000143001F021BF00004FF0FF33143001F0B7
:103E50001BBF00004C3001F0F3BF00004FF0FF33F8
:103E60004C3001F0EDBF0000143001F0EFBE000057
:103E70004FF0FF31143001F0E9BE00004C3001F08A
:103E8000BFBF00004FF0FF324C3001F0B9BF00005F
:103E90000020704710B5D0F894341A6811780429BE
:103EA000044617D1017C022914D159795289012382
:103EB0008B4013420ED1143001F082FE024648B10D
:103EC000D4F894444FF4807361792068BDE81040C1
:103ED00000F072B910BD0000406BFFF7DBBF0000BF
:103EE000704700007FB5124B036000234360C0E9B8
:103EF0000233012502260F4B0574044602900193FC
:103F000000F18402294600964FF48073143001F0CA
:103F100033FE094B0294CDE9006304F523724FF49C
:103F20008073294604F14C0001F0FAFE04B070BD24
:103F300068670008D93E0008013E00080B6830227F
:103F400082F311880A7903EB820290614A7909327F
:103F500043F822008A7912B103EB820398610223AD
:103F6000C0F894140374002080F311887047000097
:103F700038B5037F044613B190F85430ABB9201D17
:103F800001250221FFF734FF04F1140025776FF0BB
:103F9000010100F079FC84F8545004F14C006FF0FA
:103FA0000101BDE8384000F06FBC38BD10B50121FB
:103FB00004460430FFF71CFF0023237784F85430B5
:103FC00010BD000038B504460025143001F0ECFDAA
:103FD00004F14C00257701F0BBFE201D84F85450FD
:103FE0000121FFF705FF2046BDE83840FFF752BF2B
:103FF00090F8443003F06003202B07D190F845205F
:10400000212A4FF0000303D81F2A06D8002070474A
:10401000222AFBD1C0E90E3303E0034A8263072260
:10402000C2630364012070471D23002037B5D0F818
:1040300094341A681178042904461AD1017C0229A3
:1040400017D11979128901238B40134211D100F144
:104050004C05284601F03CFF58B101A9284601F063
:1040600083FED4F89444019B21790246206800F035
:10407000B5F803B030BD0000F0B500EB810385B0AA
:104080009E6904460D46FEB1302383F3118804EB8C
:104090008507301D0821FFF7ABFEFB685B691B68D5
:1040A00006F14C001BB1019001F06CFE019803A9D0
:1040B00001F05AFE024648B1039B2946204600F013
:1040C0008DF8002383F3118805B0F0BDFB685A69B1
:1040D0001268002AF5D01B8A013B1340F1D104F18C
:1040E0004402EAE7093138B550F82140DCB1302309
:1040F00083F31188D4F894241368527903EB820374
:10410000DB689B695D6845B104216018FFF770FEAC
:10411000294604F1140001F05DFD2046FFF7BAFEC8
:10412000002383F3118838BD7047000001F0D2B836
:10413000012303700023C0E90133C361836203627A
:10414000C36243620363704738B50446302383F388
:1041500011880025C0E90355C0E90555416001F00B
:10416000C9F80223237085F31188284638BD000062
:1041700070B500EB810305465069DA600E461446BF
:1041800018B110220021FDF78FFBA06918B1102291
:104190000021FDF789FB31462846BDE8704001F05B
:1041A00073B90000826802F0011282600022C0E947
:1041B0000422826101F0F4B9F0B400EB8104478974
:1041C000E4680125A4698D403D43458123600023B7
:1041D000A2606360F0BC01F00FBA0000F0B400EB25
:1041E00081040789E468012564698D403D430581A8
:1041F00023600023A2606360F0BC01F089BA000074
:1042000070B50223002504460370C0E90255C0E9D9
:104210000455C564856180F8345001F0D1F86368B5
:104220001B6823B129462046BDE87040184770BD81
:104230000378052B10B504460AD080F850300523CA
:10424000037043681B680BB1042198470023A360E7
:1042500010BD00000178052906D190F85020436870
:1042600002701B6803B118477047000070B590F8E2
:104270003430044613B1002380F8343004F1440292
:10428000204601F0AFF963689B68B3B994F84430F5
:1042900013F0600535D00021204601F04FFC0021CD
:1042A000204601F041FC63681B6813B106212046DB
:1042B0009847062384F8343070BD2046984700287C
:1042C000E4D0B4F84A30E26B9A4288BFE36394F9D1
:1042D0004430E56B002B4FF0300380F20381002D5A
:1042E00000F0F280092284F8342083F31188002141
:1042F000D4E90E232046FFF771FF002383F31188D2
:10430000DAE794F8452003F07F0343EA022340F202
:104310000232934200F0C58021D8B3F5807F48D0A7
:104320000DD8012B3FD0022B00F09380002BB2D18F
:1043300004F14C02A2630222E2632364C1E7B3F5F5
:10434000817F00F09B80B3F5407FA4D194F8463084
:10435000012BA0D1B4F84C3043F0020332E0B3F5A6
:10436000006F4DD017D8B3F5A06F31D0A3F5C0635F
:10437000012B90D8636894F846205E6894F8471043
:10438000B4F848302046B047002884D04368A3637F
:104390000368E3631AE0B3F5106F36D040F60242CB
:1043A00093427FF478AF5C4BA3630223E363002363
:1043B000C3E794F84630012B7FF46DAFB4F84C306E
:1043C00023F00203C4E90E55A4F84C30256478E7C5
:1043D000B4F84430B3F5A06F0ED194F8463084F8A9
:1043E0004E30204601F044F863681B6813B1012188
:1043F00020469847032323700023C4E90E339CE72B
:1044000004F14F03A3630123C3E72378042B10D1E6
:10441000302383F311882046FFF7C4FE85F311880B
:104420000321636884F84F5021701B680BB120464C
:10443000984794F84630002BDED084F84F300423A0
:10444000237063681B68002BD6D002212046984752
:10445000D2E794F848301D0603F00F0120460AD534
:1044600001F0B2F8012804D002287FF414AF2B4BDE
:104470009AE72B4B98E701F099F8F3E794F8463068
:10448000002B7FF408AF94F8483013F00F01B3D03D
:104490001A06204602D501F065FBADE701F058FB96
:1044A000AAE794F84630002B7FF4F5AE94F8483034
:1044B00013F00F01A0D01B06204602D501F03EFBF1
:1044C0009AE701F031FB97E7142284F8342083F354
:1044D00011882B462A4629462046FFF76DFE85F3B4
:1044E0001188E9E65DB1152284F8342083F3118840
:1044F0000021D4E90E232046FFF75EFEFDE60B22E5
:1045000084F8342083F311882B462A462946204616
:10451000FFF764FEE3E700BF9867000890670008B4
:104520009467000838B590F834300446002B3ED02C
:10453000063BDAB20F2A34D80F2B32D8DFE803F06B
:104540003731310822323131313131313131373780
:10455000C56BB0F84A309D4214D2C3681B8AB5FBC4
:10456000F3F203FB12556DB9302383F311882B4608
:104570002A462946FFF732FE85F311880A2384F87C
:1045800034300EE0142384F83430302383F3118860
:1045900000231A4619462046FFF70EFE002383F338
:1045A000118838BD036C03B198470023E7E7002169
:1045B000204601F0C3FA0021204601F0B5FA6368F5
:1045C0001B6813B10621204698470623D7E7000051
:1045D00010B590F83430142B044629D017D8062B88
:1045E00005D001D81BB110BD093B022BFBD800211F
:1045F000204601F0A3FA0021204601F095FA6368F5
:104600001B6813B1062120469847062319E0152B95
:10461000E9D10B2380F83430302383F31188002351
:104620001A461946FFF7DAFD002383F31188DAE70B
:10463000C3689B695B68002BD5D1036C03B19847B5
:10464000002384F83430CEE70023037582680369C1
:104650001B6899689142FBD25A68036042601060FF
:104660005860704700230375826803691B68996866
:104670009142FBD85A6803604260106058607047EE
:1046800008B50846302383F311880B7D032B05D032
:10469000042B0DD02BB983F3118808BD8B69002240
:1046A0001A604FF0FF338361FFF7CEFF0023F2E77C
:1046B000D1E9003213605A60F3E70000FFF7C4BF8E
:1046C000054BD9680875186802681A6053600122A2
:1046D0000275D860FBF71EBE485C002030B50C4B5D
:1046E000DD684B1C87B004460FD02B46094A68464C
:1046F00000F05EF92046FFF7E3FF009B13B1684628
:1047000000F060F9A86907B030BDFFF7D9FFF9E7FD
:10471000485C002081460008044B1A68DB689068FA
:104720009B68984294BF002001207047485C00209D
:10473000084B10B51C68D86822681A6053600122C3
:104740002275DC60FFF78EFF01462046BDE8104071
:10475000FBF7E0BD485C002038B5074C0749084826
:10476000012300252370656001F0EAFB022323701A
:1047700085F3118838BD00BFB05E0020A067000837
:10478000485C002008B572B6044B186500F048FC80
:1047900000F0FEFC024B03221A70FEE7485C00208A
:1047A000B05E002000F044B9034A516853685B1AB8
:1047B0009842FBD8704700BF001000E08B600223D6
:1047C00008618B82084670478368A3F1840243F82E
:1047D000142C026943F8442C426943F8402C094ADE
:1047E00043F8242CC26843F8182C022203F80C2C3E
:1047F000002203F80B2C044A43F8102CA3F12000EC
:10480000704700BF2D030008485C002008B5FFF783
:10481000DBFFBDE80840FFF751BF0000024BDB683B
:1048200098610F20FFF74CBF485C0020302383F3D2
:104830001188FFF7F3BF000008B50146302383F36A
:1048400011880820FFF74AFF002383F3118808BD71
:10485000064BDB6839B1426818605A6013604360E8
:104860000420FFF73BBF4FF0FF307047485C00204B
:104870000368984206D01A68026050609961184631
:10488000FFF71CBF7047000038B504460D4620688E
:10489000844200D138BD036823605C608561FFF706
:1048A0000DFFF4E710B503689C68A2420CD85C6861
:1048B0008A600B604C602160596099688A1A9A601E
:1048C0004FF0FF33836010BD1B68121BECE7000044
:1048D0000A2938BF0A2170B504460D460A26601918
:1048E00001F028FB01F014FB041BA54203D8751C42
:1048F0002E460446F3E70A2E04D9BDE87040012095
:1049000001F05EBB70BD0000F8B5144B0D46D961D7
:1049100003F1100141600A2A1969826038BF0A2236
:10492000016048601861A818144601F0F5FA0A27DA
:1049300001F0EEFA431BA342064606D37C1C28195D
:1049400001F0F8FA27463546F2E70A2F04D9BDE808
:10495000F840012001F034BBF8BD00BF485C0020E6
:10496000F8B506460D4601F0D3FA0F4A134653F840
:10497000107F9F4206D12A4601463046BDE8F840E6
:10498000FFF7C2BFD169BB68441A2C1928BF2C4657
:10499000A34202D92946FFF79BFF2246314603482E
:1049A000BDE8F840FFF77EBF485C0020585C00205F
:1049B00010B4C0E9032300235DF8044B4361FFF703
:1049C000CFBF000010B5194C236998420DD0D0E933
:1049D0000032816813605A609A680A449A60002322
:1049E00003604FF0FF33A36110BD2346026843F814
:1049F000102F53600022026022699A4203D1BDE861
:104A0000104001F091BA936881680B44936001F003
:104A10007FFA2269E1699268441AA242E4D91144FA
:104A2000BDE81040091AFFF753BF00BF485C0020E3
:104A30002DE9F047DFF8BC8008F110072C4ED8F8BC
:104A4000105001F065FAD8F81C40AA68031B9A427E
:104A50003ED81444D5E900324FF00009C8F81C4094
:104A600013605A60C5F80090D8F81030B34201D1F5
:104A700001F05AFA89F31188D5E90331284698479D
:104A8000302383F311886B69002BD8D001F040FAF2
:104A90006A69A0EB04094A4582460DD2022001F062
:104AA0008FFA0022D8F81030B34208D15146284678
:104AB000BDE8F047FFF728BF121A2244F2E712EBD5
:104AC000090938BF4A4629463846FFF7EBFEB5E7E5
:104AD000D8F81030B34208D01444211AC8F81C008A
:104AE000A960BDE8F047FFF7F3BEBDE8F08700BF5F
:104AF000585C0020485C002038B501F009FA054AEE
:104B0000D2E90845031B181945F10001C2E9080163
:104B100038BD00BF485C002000207047FEE7000061
:104B2000704700004FF0FF307047000002290CD0A2
:104B3000032904D00129074818BF00207047032A21
:104B400005D8054800EBC2007047044870470020B4
:104B5000704700BF786800082C2300202C680008EC
:104B600070B59AB00546084601A9144600F0C2F88F
:104B700001A8FCF791FE431C5B00C5E9003400224C
:104B8000237003236370C6B201AB02341046D1B266
:104B90008E4204F1020401D81AB070BD13F8011B53
:104BA00004F8021C04F8010C0132F0E708B53023C8
:104BB00083F311880348FFF739FA002383F3118840
:104BC00008BD00BFB85E002090F8443003F01F021B
:104BD000012A07D190F845200B2A03D10023C0E910
:104BE0000E3315E003F06003202B08D1B0F84830F5
:104BF0002BB990F84520212A03D81F2A04D8FFF7A3
:104C0000F7B9222AEBD0FAE7034A82630722C2638C
:104C100003640120704700BF2423002007B5052945
:104C200017D8DFE801F0191603191920302383F390
:104C30001188104A01900121FFF79AFA01980E4A53
:104C40000221FFF795FA0D48FFF7BCF9002383F323
:104C5000118803B05DF804FB302383F31188074803
:104C6000FFF786F9F2E7302383F311880348FFF753
:104C70009DF9EBE7CC670008F0670008B85E0020FC
:104C800038B50C4D0C4C0D492A4604F10800FFF7CD
:104C900067FF05F1CA0204F110000949FFF760FF40
:104CA00005F5CA7204F118000649BDE83840FFF75F
:104CB00057BF00BF806300202C230020AC67000892
:104CC000B6670008C167000870B5044608460D467F
:104CD000FCF7E2FDC6B22046013403780BB9184652
:104CE00070BD32462946FCF7C3FD0028F3D10120F0
:104CF000F6E700002DE9F84F05460C46FCF7CCFD21
:104D00002B49C6B22846FFF7DFFF08B10536F6B2D9
:104D100028492846FFF7D8FF08B11036F6B2632EAF
:104D20000DD8DFF88C80DFF88C90234FDFF890A04F
:104D3000DFF890B02E7846B92670BDE8F88F294686
:104D40002046BDE8F84F01F089BC252E2BD1072263
:104D500041462846FCF78CFD58B9DBF8003023604B
:104D6000DBF804306360DBF80830A36007350C34EF
:104D7000E0E7082249462846FCF77AFD98B90F4B30
:104D8000A21C197809090232C95D02F8041C13F843
:104D9000011B01F00F015345C95D02F8031CF0D15E
:104DA00018340835C6E704F8016B0135C2E700BFC7
:104DB00098680008C1670008AD680008107AFF1FF6
:104DC0001C7AFF1FA0680008BFF34F8F024AD36808
:104DD000DB03FCD4704700BF003C024008B5094B20
:104DE0001B7873B9FFF7F0FF074B1A69002ABFBFA2
:104DF000064A5A6002F188325A601A6822F48062C8
:104E00001A6008BDDE650020003C024023016745B2
:104E100008B50B4B1B7893B9FFF7D6FF094B1A69FE
:104E200042F000421A611A6842F480521A601A680D
:104E300022F480521A601A6842F480621A6008BD37
:104E4000DE650020003C02400728F0B516D80C4C67
:104E50000C4923787BB90C4D0E4608234FF00062B5
:104E600055F8047B46F8042B013B13F0FF033A444A
:104E7000F6D10123237051F82000F0BD0020FCE79B
:104E800000660020E0650020C0680008014B53F870
:104E900020007047C068000808207047072810B538
:104EA000044601D9002010BDFFF7CEFF064B53F892
:104EB00024301844C21A0BB90120F4E712680132F9
:104EC000F0D1043BF6E700BFC0680008072810B522
:104ED000044621D8FFF778FFFFF780FF0F4AF3233E
:104EE000D360C300DBB243F4007343F002031361E9
:104EF000136943F480331361FFF766FFFFF7A4FFE4
:104F0000074B53F8241000F03FF9FFF781FF2046CC
:104F1000BDE81040FFF7C2BF002010BD003C0240BA
:104F2000C0680008F8B512F00103144642D1851894
:104F30002E4A954257D82E4B1B6813F0010352D0CE
:104F40002C4DFFF74BFFF323EB60FFF73DFF40F2E3
:104F50000127032C15D824F001046618254C401AAB
:104F600040F20117B142236900EB010524D123F07F
:104F700001032361FFF74CFF0120F8BD043C04301E
:104F8000E7E78307E7D12B6923F440732B612B6993
:104F90003B432B6151F8046B0660BFF34F8FFFF763
:104FA00013FF03689E42E9D02B6923F001032B61B4
:104FB000FFF72EFF0020E0E723F44073236123690D
:104FC0003B4323610B882B80BFF34F8FFFF7FCFE21
:104FD0002D8831F8023BADB2AB42C3D0236923F038
:104FE00001032361E4E71846C7E700BF0000080893
:104FF00000380240003C0240084908B50B7828B14F
:105000001BB9FFF7EBFE01230B7008BD002BFCD092
:10501000BDE808400870FFF7FBBE00BFDE6500205A
:1050200008B50649064800F0B1F8BDE808404FF45D
:1050300080314FF0805000F0A9B800BF00FF0100A0
:10504000000100200846114601F06CBA012001F071
:1050500069BA0000084601F083BA000038B5EFF3E2
:1050600011859DB9EFF30584C4F30804302334B1EE
:1050700083F31188FFF740FD85F3118838BD83F372
:105080001188FFF739FD84F3118838BDBDE8384039
:10509000FFF732BD38B5FFF7E1FF114C114AC008E8
:1050A00040EA4170A0FB025EC908A0FB040C1CEBA7
:1050B000050CA1FB04404FF000035B41A1FB021271
:1050C0001CEB040C43EB000011EB0E0142F100025B
:1050D000411842F10000090941EA007038BD00BFE3
:1050E000CFF753E3A59BC42010B50244064BD2B2C0
:1050F000904200D110BD441C00B253F8200041F88A
:10510000040BE0B2F4E700BF502800400F4B30B56D
:105110001C6F240407D41C6F44F400741C671C6FBC
:1051200044F400441C670A4C236843F480732360F2
:105130000244084BD2B2904200D130BD441C00B2B0
:1051400051F8045B43F82050E0B2F4E70038024025
:10515000007000405028004007B5012201A900203E
:10516000FFF7C2FF019803B05DF804FB13B50446D6
:10517000FFF7F2FFA04205D0012201A9002001940F
:10518000FFF7C4FF02B010BD704700007047000079
:1051900070470000074B45F255521A6002225A60D0
:1051A00040F6FF729A604CF6CC421A60024B012224
:1051B0001A7070470030004008660020034B1B78CF
:1051C0001BB1034B4AF6AA221A60704708660020FA
:1051D00000300040034B1A681AB9034AD2F8742809
:1051E0001A6070470466002000300240024B4FF006
:1051F0008072C3F8742870470030024008B5FFF78A
:10520000E9FF024B1868C0F3407008BD0466002037
:1052100008B5FFF7DFFF024B1868C0F3007008BD48
:105220000466002070470000FEE700000A4B0B48B0
:105230000B4A90420BD30B4BDA1C121AC11E22F000
:1052400003028B4238BF00220021FCF72DBB53F82C
:10525000041B40F8041BECE7C86A00080C67002038
:105260000C6700200C67002070B5D0E915439E68DC
:1052700000224FF0FF3504EB42135101D3F800092F
:105280000028BEBFD3F8000940F08040C3F80009F1
:10529000D3F8000B0028BEBFD3F8000B40F08040CD
:1052A000C3F8000B013263189642C3F80859C3F8DB
:1052B000085BE0D24FF00113C4F81C3870BD000049
:1052C000890141F02001016103699B06FCD4122091
:1052D000FFF76ABA10B5054C2046FEF729FF4FF0DC
:1052E000A0436365024BA36510BD00BF0C660020A0
:1052F0000469000870B50378012B054650D12A4B8C
:10530000446D98421BD1294B5A6B42F080025A637C
:105310005A6D42F080025A655A6D5A6942F0800215
:105320005A615A6922F080025A610E2143205B695A
:10533000FEF748FD1E4BE3601E4BC4F80038002307
:10534000C4F8003EC02323606E6D4FF40413A363C2
:105350003369002BFCDA012333610C20FFF724FAB8
:105360003369DB07FCD41220FFF71EFA3369002BE8
:10537000FCDA0026A6602846FFF776FF6B68C4F8C3
:105380001068DB68C4F81468C4F81C684BB90A4B91
:10539000A3614FF0FF336361A36843F00103A3608F
:1053A00070BD064BF4E700BF0C66002000380240D9
:1053B0004014004003002002003C30C0083C30C0D4
:1053C000F8B5446D054600212046FFF779FFA96D29
:1053D00000234FF001128F68C4F834384FF0006694
:1053E000C4F81C284FF0FF3004EB431201339F42F6
:1053F000C2F80069C2F8006BC2F80809C2F8080BCD
:10540000F2D20B686A6DEB65636210231361166953
:1054100016F01006FBD11220FFF7C6F9D4F80038B9
:1054200023F4FE63C4F80038A36943F4402343F037
:105430001003A3610923C4F81038C4F814380A4BC8
:10544000EB604FF0C043C4F8103B084BC4F8003B7E
:10545000C4F81069C4F80039EB6D03F1100243F48D
:105460008013EA65A362F8BDE06800084080001080
:10547000426D90F84E10D2F8003823F4FE6343EAF0
:105480000113C2F8003870472DE9F84300EB81039F
:10549000456DDA68166806F00306731E022B05EBED
:1054A00041130C4680460FFA81F94FEA41104FF044
:1054B0000001C3F8101B4FF0010104F1100398BF65
:1054C000B60401FA03F391698EBF334E06F180569C
:1054D00006F5004600293AD0578A04F158014901DF
:1054E00037436F50D5F81C180B43C5F81C382B18E0
:1054F0000021C3F8101953690127611EA7409BB30F
:10550000138A928B9B08012A88BF5343D8F85C20EA
:10551000981842EA034301F1400205EB8202C8F801
:105520005C00214653602846FFF7CAFE08EB89005D
:10553000C3681B8A43EA8453483464011E432E51D6
:10554000D5F81C381F43C5F81C78BDE8F88305EB77
:105550004917D7F8001B21F40041C7F8001BD5F804
:105560001C1821EA0303C0E704F13F0305EB8303A2
:105570000A4A5A6028462146FFF7A2FE05EB491069
:10558000D0F8003923F40043C0F80039D5F81C38AE
:1055900023EA0707D7E700BF0080001000040002DD
:1055A000826D1268C265FFF75FBE00005831436D1F
:1055B00049015B5813F4004004D013F4001F0CBFE2
:1055C00002200120704700004831436D49015B58BB
:1055D00013F4004004D013F4001F0CBF022001207C
:1055E0007047000000EB8101CB68196A0B681360FB
:1055F0004B6853607047000000EB810330B5DD68F5
:10560000AA691368D36019B9402B84BF4023136083
:105610006B8A1468426D1C44013CB4FBF3F4634391
:10562000033323F0030302EB411043EAC44343F086
:10563000C043C0F8103B2B6803F00303012B09B2F1
:105640000ED1D2F8083802EB411013F4807FD0F865
:10565000003B14BF43F0805343F00053C0F8003BBD
:1056600002EB4112D2F8003B43F00443C2F8003B86
:1056700030BD00002DE9F041244D6E6D06EB401366
:105680000446D3F8087BC3F8087B38070AD5D6F858
:105690001438190706D505EB84032146DB68284634
:1056A0005B689847FA071FD5D6F81438DB071BD577
:1056B00005EB8403D968CCB98B69488A5A68B2FB78
:1056C000F0F600FB16228AB91868DA6890420DD20B
:1056D000121AC3E90024302383F311880B482146B2
:1056E000FFF78AFF84F31188BDE8F081012303FAF4
:1056F00004F26B8923EA02036B81CB68002BF3D0A1
:1057000021460248BDE8F041184700BF0C66002062
:1057100000EB810370B5DD68436D6C692668E66057
:105720004A0156BB1A444FF40020C2F810092A68F7
:1057300002F00302012A0AB20ED1D3F8080803EBE3
:10574000421410F4807FD4F8000914BF40F0805058
:1057500040F00050C4F8000903EB4212D2F80009EF
:1057600040F00440C2F80009D3F83408012202FADC
:1057700001F10143C3F8341870BD19B9402E84BF3C
:105780004020206020682E8A8419013CB4FBF6F486
:1057900040EAC44040F000501A44C6E72DE9F843FF
:1057A0003B4D6E6D06EB40130446D3F80889C3F8F1
:1057B000088918F0010F4FEA40171AD0D6F81038B0
:1057C000DB0716D505EB8003D9684B691868DA68E2
:1057D000904230D2121A4FF000091A60C3F80490B8
:1057E000302383F3118821462846FFF791FF89F380
:1057F000118818F0800F1CD0D6F834380126A64046
:10580000334216D005EB84036D6DD3F80CC0DCF881
:1058100014200134E4B2D2F800E005EB04342F4444
:105820005168714515D3D5F8343823EA0606C5F812
:105830003468BDE8F883012303FA04F22B8923EAD4
:1058400002032B818B68002BD3D021462846984732
:10585000CFE7BCF81000AEEB0103834228BF03463C
:10586000D7F8180980B2B3EB800FE2D89068A0F1A6
:10587000040959F8048FC4F80080A0EB0908984483
:10588000B8F1040FF5D818440B4490605360C7E793
:105890000C6600202DE9F74FA24C656D6E69AB696F
:1058A0001E4016F480586E6107D02046FEF7A8FC13
:1058B00003B0BDE8F04FFEF75BBA002E12DAD5F860
:1058C000003E98489B071EBFD5F8003E23F0030317
:1058D000C5F8003ED5F8043823F00103C5F80438B4
:1058E000FEF7B8FC370505D58E48FFF7BDFC8D489F
:1058F000FEF79EFCB0040CD5D5F8083813F0060F5F
:10590000EB6823F470530CBF43F4105343F4A053DB
:10591000EB6031071BD56368DB681BB9AB6923F00B
:105920000803AB612378052B0CD1D5F8003E7D48E8
:105930009A071EBFD5F8003E23F00303C5F8003ECA
:10594000FEF788FC6368DB680BB176489847F30282
:1059500074D4B70227D5D4F85490DFF8C8B1002723
:105960004FF0010A09EB4712D2F8003B03F4402341
:10597000B3F5802F11D1D2F8003B002B0DDA6289EC
:105980000AFA07F322EA0303638104EB8703DB6867
:10599000DB6813B1394658469847A36D01379B68B9
:1059A000FFB29F42DED9F00617D5676D3A6AC2F39F
:1059B0000A1002F00F0302F4F012B2F5802F00F08B
:1059C0008580B2F5402F08D104EB83030022DB6809
:1059D0001B6A07F5805790426AD13003D5F8184802
:1059E00013D5E10302D50020FFF744FEA20302D540
:1059F0000120FFF73FFE630302D50220FFF73AFEC6
:105A0000270302D50320FFF735FE75037FF550AF5E
:105A1000E00702D50020FFF7C1FEA10702D5012053
:105A2000FFF7BCFE620702D50220FFF7B7FE23078F
:105A30007FF53EAF0320FFF7B1FE39E7636DDFF876
:105A4000E4A0019300274FF00109A36D9B685FFA62
:105A500087FB9B453FF67DAF019B03EB4B13D3F8D0
:105A6000001901F44021B1F5802F1FD1D3F800199E
:105A700000291BDAD3F8001941F09041C3F800194E
:105A8000D3F800190029FBDB5946606DFFF718FCBD
:105A9000218909FA0BF321EA0303238104EB8B0329
:105AA000DB689B6813B15946504698470137CCE7ED
:105AB000910708BFD7F80080072A98BF03F8018B29
:105AC00002F1010298BF4FEA182884E7023304EB81
:105AD000830207F580575268D2F818C0DCF8082016
:105AE000DCE9001CA1EB0C0C002188420AD104EB7C
:105AF000830463689B699A6802449A605A68024406
:105B00005A606AE711F0030F08BFD7F800808C4590
:105B100088BF02F8018B01F1010188BF4FEA182804
:105B2000E3E700BF0C660020436D03EB4111D1F8A1
:105B3000003B43F40013C1F8003B7047436D03EB97
:105B40004111D1F8003943F40013C1F8003970470E
:105B5000436D03EB4111D1F8003B23F40013C1F86E
:105B6000003B7047436D03EB4111D1F8003923F43A
:105B70000013C1F80039704730B5039C017204333B
:105B800004FB0325C0E90653049B03630021059B26
:105B9000C160C0E90000C0E90422C0E90842C0E9D0
:105BA0000A11436330BD0000416A0022C0E90411BC
:105BB000C0E90A22C2606FF00101FEF765BE000075
:105BC000D0E90432934201D1C2680AB9181D704766
:105BD0000020704703691960C2680132C260C2695F
:105BE000134482690361934224BF436A0361002125
:105BF000FEF73EBE38B504460D46E3683BB1626928
:105C0000131D1268A3621344E362002007E0237AA5
:105C100033B929462046FEF71BFE0028EDDA38BDD1
:105C20006FF00100FBE70000C368C269013BC3607D
:105C30004369134482694361934224BF436A4361C9
:105C400000238362036B03B11847704770B530239C
:105C5000044683F31188866A3EB9FFF7CBFF0546F9
:105C600018B186F31188284670BDA36AE26A13F85A
:105C7000015BA362934202D32046FFF7D5FF0023C6
:105C800083F31188EFE700002DE9F84F04460E4634
:105C9000174698464FF0300989F311880025AA4627
:105CA000D4F828B0BBF1000F09D141462046FFF7D8
:105CB000A1FF20B18BF311882846BDE8F88FD4E905
:105CC0000A12A7EB050B521A934528BF9346BBF166
:105CD000400F1BD9334601F1400251F8040B43F841
:105CE000040B9142F9D1A36A40334036A362403598
:105CF000D4E90A239A4202D32046FFF795FF8AF39C
:105D00001188BD42D8D289F31188C9E730465A4676
:105D1000FBF7A4FDA36A5B445E44A3625D44E7E72E
:105D200010B5029C0172043303FB0421C0E9061381
:105D30000023C0E90A33039B0363049BC460C0E9EA
:105D40000000C0E90422C0E90842436310BD00001E
:105D5000026AC260426AC0E904220022C0E90A2243
:105D60006FF00101FEF790BDD0E904239A4201D102
:105D7000C26822B9184650F8043B0B6070470023F4
:105D80001846FAE7C368C2690133C3604369134424
:105D900082694361934224BF436A43610021FEF755
:105DA00067BD000038B504460D46E3683BB1236982
:105DB0001A1DA262E2691344E362002007E0237A1D
:105DC00033B929462046FEF743FD0028EDDA38BDF9
:105DD0006FF00100FBE7000003691960C268013A37
:105DE000C260C269134482690361934224BF436A5B
:105DF000036100238362036B03B1184770470000FF
:105E000070B530230D460446114683F31188866A27
:105E10002EB9FFF7C7FF10B186F3118870BDA36AD2
:105E20001D70A36AE26A01339342A36204D3E1695D
:105E300020460439FFF7D0FF002080F31188EDE7FA
:105E40002DE9F84F04460D46904699464FF0300A2A
:105E50008AF311880026B346A76A4FB949462046FF
:105E6000FFF7A0FF20B187F311883046BDE8F88F17
:105E7000D4E90A073A1AA8EB0607974228BF174643
:105E8000402F1BD905F1400355F8042B40F8042B93
:105E90009D42F9D1A36A4033A3624036D4E90A2374
:105EA0009A4204D3E16920460439FFF795FF8BF34A
:105EB00011884645D9D28AF31188CDE729463A465A
:105EC000FBF7CCFCA36A3B443D44A3623E44E5E7B8
:105ED000D0E904239A4217D1C3689BB1836A8BB17E
:105EE000043B9B1A0ED01360C368013BC360C369B7
:105EF0001A44836902619A4224BF436A0361002302
:105F000083620123184670470023FBE700F0D2B8F4
:105F10004FF08043586A70474FF080430022586327
:105F20001A610222DA6070474FF080430022DA6083
:105F3000704700004FF0804358637047FEE7000051
:105F400070B51B4B01630025044686B0586085621E
:105F50000E46FDF7E9FE04F11003C4E904334FF0E7
:105F6000FF33C4E90635C4E90044A560E562FFF7E4
:105F7000CFFF2B460246C4E9082304F134010D4A41
:105F8000256580232046FEF719FC0123E0600A4ABC
:105F90000375009272680192B268CDE90223074B43
:105FA0006846CDE90435FEF731FC06B070BD00BF90
:105FB000B05E002010690008156900083D5F000808
:105FC000024AD36A1843D062704700BF485C002081
:105FD0004B6843608B688360CB68C3600B69436127
:105FE0004B6903628B6943620B6803607047000072
:105FF00008B5264B26481A6940F2FF110A431A6178
:106000001A6922F4FF7222F001021A611A691A6BEE
:106010000A431A631A6D0A431A651E4A1B6D11461C
:10602000FFF7D6FF02F11C0100F58060FFF7D0FFFB
:1060300002F1380100F58060FFF7CAFF02F1540158
:1060400000F58060FFF7C4FF02F1700100F5806089
:10605000FFF7BEFF02F18C0100F58060FFF7B8FF8B
:1060600002F1A80100F58060FFF7B2FF02F1C40160
:1060700000F58060FFF7ACFF02F1E00100F5806001
:10608000FFF7A6FFBDE8084000F090B800380240D6
:10609000000002401C69000808B500F0FBF9FEF79B
:1060A0005BFBFFF797F8BDE80840FEF7E9BD00008D
:1060B000704700000F4B1A6C42F001021A641A6E0E
:1060C00042F001021A660C4A1B6E936843F001030A
:1060D00093604FF0804353229A624FF0FF32DA62AE
:1060E00000229A615A63DA605A6001225A611A608A
:1060F000704700BF00380240002004E04FF08042AB
:1061000008B51169D3680B40D9B2C9439B07116127
:1061100007D5302383F31188FEF744FB002383F374
:10612000118808BD1F4B1A696FEAC2526FEAD2523A
:106130001A611A69C2F308021A614FF0FF301A6936
:106140005A69586100215A6959615A691A6A62F09C
:1061500080521A621A6A02F080521A621A6A5A6AE5
:1061600058625A6A59625A6A1A6C42F080521A642A
:106170001A6E42F080521A661A6E0B4A106840F48A
:1061800080701060186F00F44070B0F5007F1EBF83
:106190004FF4803018671967536823F40073536015
:1061A00000F054B90038024000700040334B4FF00B
:1061B00080521A64324A4FF4404111601A6842F02A
:1061C00001021A601A689107FCD59A6822F003024E
:1061D0009A602A4B9A6812F00C02FBD1196801F000
:1061E000F90119609A601A6842F480321A601A68DC
:1061F0009203FCD55A6F42F001025A671F4B5A6F47
:106200009007FCD51F4A5A601A6842F080721A60E3
:106210001B4A53685904FCD5184B1A689201FCD5E7
:10622000194A9A60194B1A68194B9A42194B21D195
:10623000194A1168194A91421CD140F205121A609C
:10624000144A136803F00F03052BFAD10B4B9A681D
:1062500042F002029A609A6802F00C02082AFAD10F
:106260005A6C42F480425A645A6E42F480425A6632
:106270005B6E704740F20572E1E700BF00380240F4
:10628000007000400854400700948838002004E063
:1062900011640020003C024000ED00E041C20F41CB
:1062A000074A08B5536903F00103536123B1054A56
:1062B00013680BB150689847BDE80840FDF758BD1A
:1062C000003C014084660020074A08B5536903F08A
:1062D0000203536123B1054A93680BB1D068984714
:1062E000BDE80840FDF744BD003C01408466002045
:1062F000074A08B5536903F00403536123B1054A03
:1063000013690BB150699847BDE80840FDF730BDEF
:10631000003C014084660020074A08B5536903F039
:106320000803536123B1054A93690BB1D0699847BB
:10633000BDE80840FDF71CBD003C0140846600201C
:10634000074A08B5536903F01003536123B1054AA6
:10635000136A0BB1506A9847BDE80840FDF708BDC5
:10636000003C014084660020164B10B55C6904F4C3
:1063700078725A61A30604D5134A936A0BB1D06AA6
:106380009847600604D5104A136B0BB1506B9847C1
:10639000210604D50C4A936B0BB1D06B9847E205EC
:1063A00004D5094A136C0BB1506C9847A30504D56A
:1063B000054A936C0BB1D06C9847BDE81040FDF7CF
:1063C000D7BC00BF003C014084660020194B10B5CB
:1063D0005C6904F47C425A61620504D5164A136D67
:1063E0000BB1506D9847230504D5134A936D0BB13B
:1063F000D06D9847E00404D50F4A136E0BB1506E70
:106400009847A10404D50C4A936E0BB1D06E9847FF
:10641000620404D5084A136F0BB1506F98472304E8
:1064200004D5054A936F0BB1D06F9847BDE8104073
:10643000FDF79EBC003C01408466002008B5FFF7D4
:106440005DFEBDE80840FDF793BC0000062108B5DD
:106450000846FDF7B7FC06210720FDF7B3FC06212F
:106460000820FDF7AFFC06210920FDF7ABFC062153
:106470000A20FDF7A7FC06211720FDF7A3FC062143
:106480002820FDF79FFCBDE8084007211C20FDF7F0
:1064900099BC000008B5FFF745FE00F00BF8FDF7CA
:1064A00045FEFDF71DFDFFF703FEBDE80840FFF7C1
:1064B0002DBD00000023054A19460133102BC2E907
:1064C000001102F10802F8D1704700BF8466002075
:1064D0000B460146184600F02DB8000000F040B809
:1064E000012838BF012010B50446204600F030F8DE
:1064F00030B900F007F808B900F00CF88047F4E76D
:1065000010BD0000024B1868BFF35B8F704700BFDF
:106510000467002008B5062000F084F80120FEF78B
:10652000FDFA0000024B0A4601461868FEF78ABDD4
:106530004C23002010B5054C13462CB10A460146E9
:106540000220AFF3008010BD2046FCE700000000F1
:10655000024B01461868FEF779BD00BF4C230020AE
:10656000024B01461868FEF775BD00BF4C230020A2
:1065700010B501390244904201D1002005E00378B2
:1065800011F8014FA34201D0181B10BD0130F2E7F2
:106590002DE9F041A3B1C91A17780144044603F16B
:1065A000FF3C8C42204601D9002009E00578BD421D
:1065B00004F10104F5D10CEB0405D618A54201D174
:1065C000BDE8F08115F8018D16F801EDF045F5D024
:1065D000E7E700001F2938B504460D4604D9162305
:1065E00003604FF0FF3038BD426C12B152F82130D9
:1065F0004BB9204600F030F82A4601462046BDE857
:10660000384000F017B8012B0AD0591C03D11623CB
:1066100003600120E7E7002442F825402846984718
:106620000020E0E7024B01461868FFF7D3BF00BF28
:106630004C23002038B5074D002304460846114678
:106640002B60FEF76FFA431C02D12B6803B1236065
:1066500038BD00BF08670020FEF75EBA034611F898
:10666000012B03F8012B002AF9D1704773772D73A2
:106670007061722D663430372D626C0053544D3387
:1066800032463F3F3F0053544D333246343078005A
:1066900053544D3332463432780053544D333246DE
:1066A00034343658580000000120330000104100F7
:1066B00001105A00031059000710310000000000BB
:1066C0007C660008130400008666000819040000B8
:1066D00090660008210400009A66000840A2E4F1D8
:1066E000646891060041A3E5F26569920700000025
:1066F0004261642043414E496661636520696E646E
:1067000065782E00000100000001FF0000640040D9
:106710000068004080000000008000000000800051
:10672000000000000000000065210008292A000880
:1067300031290008A5210008B1210008B123000873
:1067400075210008852100087921000881210008B1
:106750007D210008D5220008892100082D2D000880
:1067600099210008A9220008000000005D3E0008F1
:10677000493E0008853E0008713E00087D3E000845
:10678000693E0008553E0008413E0008913E000861
:106790000000000001000000000000006330000065
:1067A0009C670008A05C0020B05E00204172647508
:1067B00050696C6F740025424F415244252D424C64
:1067C000002553455249414C2500000002000000BD
:1067D0000000000079400008E5400008400040004B
:1067E00050630020606300200200000000000000F1
:1067F0000300000000000000294100080000000024
:106800001000000070630020000000000100000084
:10681000000000000C660020010102001D4C000871
:106820002D4B0008C94B0008AD4B00084300000089
:106830003468000809024300020100C03209040064
:1068400000010202010005240010010524010001DD
:10685000042402020524060001070582030800FF44
:1068600009040100020A00000007050102400000BF
:106870000705810240000000120000008068000847
:1068800012011001020000400912415700020102EA
:10689000030100000403090425424F41524425002E
:1068A00073772D737061722D66343037003031325A
:1068B00033343536373839414243444546000000C9
:1068C00000400000004000000040000000400000C8
:1068D00000000100000002000000020000000200B1
:1068E000000000006D42000825450008D145000861
:1068F000400040006C6600206C6600200100000033
:106900007C660020800000004001000003000000C1
:106910006D61696E0069646C650000000000802A8A
:1069200000000000AAAAAAAA00000024FFFF00009D
:106930000000000000A00A00006800000000000045
:10694000AA6AAAAA000000007FFF000000009009C8
:10695000000000000000010000000000AAAAAAAA8E
:1069600000000000FFFE000000000000000000002A
:106970001A000000000000009AAAAAAA0000000065
:10698000FFFF000099000000000000000000000070
:1069900000000000AAAAAAAA00000000FFFF000051
:1069A00000000000000000000000000000000000E7
:1069B000AAAAAAAA00000000FFFF00000000000031
:1069C000000000000000000000000000AAAAAAAA1F
:1069D00000000000FFFF00000000000000000000B9
:1069E00000000000000000000A000000000000009D
:1069F0000300000000000000000000000000000094
:106A00000000000000000000000000000000000086
:106A100000000000000000007017000000000000EF
:106A2000000007000000000040420F00FE2A0100A5
:106A3000D2040000FF00960000000008009600004D
:106A40000000080004000000946800080000000036
:106A50000000000000000000000000000000000036
:106A60000000000050230020000000000000000093
:106A70000000000000000000000000000000000016
:106A80000000000000000000000000000000000006
:106A900000000000000000000000000000000000F6
:106AA00000000000000000000000000000000000E6
:106AB00000000000000000000000000000000000D6
:086AC0000000000000000000CE
:00000001FF
